:020000020000FC
:100000000C94184D189518951895189518951895DD
:100010001895189518951895189518951895189578
:100020001895189518951895189518951895189568
:100030001895189518951895189518950C94412FA2
:1000400018951895189518950C9439481895189581
:100050001895189518951895189518951895189538
:100060001895189518951895189518951895189528
:1000700018951895189518950C9413481895189577
:100080001895189518951895189518950D0A20002B
:100090000D0A0A205B434D2D352056657273696F3A
:1000A0006E20312E31325D000D0A20546F737320A3
:1000B0004D6F64650D0A000D0A202D3E5B44796E7C
:1000C000616D6978656C5D3A000D0A203C2D5B44DA
:1000D000796E616D6978656C5D3A000D0A203C2D82
:1000E0003E50433A00203C2D3E44796E616D697864
:1000F000656C3A000D0A2041726520796F75207396
:10010000757265203F28792F4E29000D0A205573FE
:10011000616765203A20476F205B506F736974698F
:100120006F6E20416E676C6528307830307E307895
:10013000336666295D000D0A20416C6C2044796E9F
:10014000616D6978656C27732049442077696C6C10
:100150002062652073657420746F20002E20417228
:100160006520796F7520737572653F28592F4E2968
:10017000000D0A204572726F72315B436865636BD4
:100180002044796E616D6978656C2056657273697B
:100190006F6E206973206D6F7265207468616E20C8
:1001A000335D000D0A2042284265666F7265292C76
:1001B0004E284E657874292C512851756974290090
:1001C0000D0A203438354D6F6E69746F72205B4CA8
:1001D000462C43522061726520616464656420612D
:1001E000742070617573652074696D655D0D0A001A
:1001F0000D0A204E6F20446174615B61742042726D
:100200006F61646361737420494420307846455DB2
:10021000000D0A204E6F20446174612843686563B5
:100220006B2049442C204F7065726174696E6720A1
:100230004D6F64652C20426175642072617465297C
:1002400000204C454E3A000D0A204C454420426C9B
:10025000696E6B2049443A002044796E616D69787B
:10026000656C7320466F756E642E000D0A204C4538
:100270004420426C696E6B2049443A000D20466F61
:10028000756E642120424155445F5245473A002C27
:100290002049443A000D0A20426175642052656786
:1002A000206973206368616E67656420746F200045
:1002B000425053000D0A2049443A30202D20000DB1
:1002C0000A2044656C61793A000D0A20546F7271FE
:1002D000756520456E61626C65000D0A204D6F7674
:1002E000652030203C2D3E203078336666000D0AB4
:1002F00020416E79204B657920746F20436F6E74B6
:10030000696E75652E2E2E000D0A205B45455052F4
:100310004F4D20415245415D0D0A204D4F44454C03
:100320005F4E554D4245525F4C202020202020201A
:1003300020285229205B000D0A204D4F44454C5F78
:100340004E554D4245525F4820202020202020203D
:10035000285229205B000D0A2056455253494F4E22
:100360002020202020202020202020202020202885
:100370005229205B000D0A20494420202020202003
:100380002020202020202020202020202028522F24
:1003900057295B000D0A20424155445F52415445A4
:1003A00020202020202020202020202028522F57CD
:1003B000295B000D0A2052455455524E5F44454C6E
:1003C00041595F54494D452020202028522F57295C
:1003D0005B000D0A2043575F414E474C455F4C4937
:1003E0004D49545F4C202020202028522F57295B54
:1003F000000D0A2043575F414E474C455F4C494D25
:1004000049545F48202020202028522F57295B0084
:100410000D0A204343575F414E474C455F4C494DC1
:1004200049545F4C2020202028522F57295B000D73
:100430000A204343575F414E474C455F4C494D4965
:10044000545F482020202028522F57295B000D0A96
:10045000202852455345525645442920202020202B
:1004600020202020202028522F57295B000D0A2011
:100470004C494D49545F54454D5045524154555295
:10048000452020202028522F57295B000D0A2044A8
:100490004F574E5F4C494D49545F564F4C5441475E
:1004A0004520202028522F57295B000D0A20555047
:1004B0005F4C494D49545F564F4C544147452020AD
:1004C00020202028522F57295B000D0A204D41582B
:1004D0005F544F525155455F4C2020202020202052
:1004E000202028522F57295B000D0A204D41585FCC
:1004F000544F525155455F48202020202020202075
:100500002028522F57295B000D0A2052455455527E
:100510004E5F4C4556454C20202020202020202096
:1005200028522F57295B000D0A20414C41524D5F44
:100530004C4544202020202020202020202020283E
:10054000522F57295B000D0A20414C41524D5F53F9
:10055000485554444F574E20202020202020285218
:100560002F57295B000D0A20285245534552564506
:100570004429202020202020202020202028522F05
:1005800057295B000D0A20444F574E5F43414C49A9
:1005900042524154494F4E5F4C20202028522F5741
:1005A000295B000D0A20444F574E5F43414C49429E
:1005B000524154494F4E5F4820202028522F57293E
:1005C0005B000D0A2055505F43414C494252415453
:1005D000494F4E5F4C202020202028522F57295B66
:1005E000000D0A2055505F43414C49425241544945
:1005F0004F4E5F48202020202028522F57295B0093
:100600000D0A205B52414D20415245415D0D0A20AB
:10061000544F525155455F454E41424C4520202094
:10062000202020202028522F57295B000D0A204C23
:100630004544202020202020202020202020202071
:100640002020202028522F57295B000D0A204357D5
:100650005F434F4D504C49414E43455F4D415247DA
:10066000494E2028522F57295B000D0A204343573B
:100670005F434F4D504C49414E43455F4D415247BA
:10068000494E28522F57295B000D0A2043575F43DC
:100690004F4D504C49414E43455F534C4F504520C0
:1006A0002028522F57295B000D0A204343575F43F0
:1006B0004F4D504C49414E43455F534C4F504520A0
:1006C00028522F57295B000D0A20474F414C5F509D
:1006D0004F534954494F4E5F4C2020202020202862
:1006E000522F57295B000D0A20474F414C5F504F56
:1006F000534954494F4E5F48202020202020285243
:100700002F57295B000D0A204D4F56494E475F5326
:10071000504545445F4C2020202020202028522F87
:1007200057295B000D0A204D4F56494E475F5350E5
:100730004545445F482020202020202028522F5764
:10074000295B000D0A20544F525155455F4C494DCD
:1007500049545F4C2020202020202028522F572948
:100760005B000D0A20544F525155455F4C494D498D
:10077000545F482020202020202028522F57295B1A
:10078000000D0A2050524553454E545F504F534977
:1007900054494F4E5F4C20202020285229205B00D6
:1007A0000D0A2050524553454E545F504F53495403
:1007B000494F4E5F4820202020285229205B000D01
:1007C0000A2050524553454E545F53504545445FAF
:1007D0004C20202020202020285229205B000D0AB8
:1007E0002050524553454E545F53504545445F4851
:1007F00020202020202020285229205B000D0A20C4
:1008000050524553454E545F4C4F41445F4C20205D
:10081000202020202020285229205B000D0A205073
:10082000524553454E545F4C4F41445F4820202071
:100830002020202020285229205B000D0A20505221
:100840004553454E545F564F4C5441474520202058
:1008500020202020285229205B000D0A20505245DC
:1008600053454E545F54454D5045524154555245A1
:10087000202020285229205B000D0A20524547499C
:100880005354455245445F494E53545255432E20CC
:100890002028522F57295B000D0A205245534552FC
:1008A0005645442850415553455F54494D452920EC
:1008B00028522F57295B000D0A204D4F56494E47AD
:1008C0002020202020202020202020202020202028
:1008D000285229205B000D0A204C4F434B2020203A
:1008E00020202020202020202020202020202852CE
:1008F0002F57295B000D0A2050554E43485F4C206E
:100900002020202020202020202020202028522F9E
:1009100057295B000D0A2050554E43485F48202060
:1009200020202020202020202020202028522F5747
:10093000295B000D0A0A2044554D50284429203ACD
:100940002044756D7020636F6E74726F6C207461DB
:10095000626C652E000D0A204944205B49445F4EBD
:10096000554D5D203A20536574204944206F662020
:1009700064796E616D6978656C2E000D0A204349BB
:1009800044205B49445F4E554D5D203A20436861E9
:100990006E676520436F6E74726F6C2049442E0041
:1009A0000D0A2052454144205B414444525D5B4C5A
:1009B000454E5D203A205265616420646174612E69
:1009C0002065782952656164203130203220285218
:1009D0006561642066726F6D20307831302C206C38
:1009E000656E677468203229000D0A2057524954F9
:1009F00045205B414444525D5B44415441315D2E8E
:100A00002E203A20577269746520646174612E202B
:100A100065782957726974652031342C3120285744
:100A20007269746520312061742030783134290076
:100A30000D0A205245475F5752205B414444525DA6
:100A40005B44415441315D2E2E203A205265676946
:100A50007374657220777269746520696E7374753A
:100A6000726374696F6E000D0A20414354494F4E02
:100A7000203A20416374696F6E205245475F575298
:100A800020696E737472756374696F6E000D0A204D
:100A9000476F205B504F534954494F4E5D5B535055
:100AA0004545445D3A20476F746F20746865207037
:100AB0006F736974696F6E207769746820746865F4
:100AC0002073706565642E000D0A20484558205B30
:100AD0004E554D5D5B4E554D5D2E2E2E203A2054C9
:100AE00072616E736D6974652072617720646174E0
:100AF000612E2065782948657820464620464620A4
:100B00003031203033000D0A205245534554203AED
:100B10002044796E616D6978656C205265736574E7
:100B20002E000D0A2050494E47205B4E554D5D3A30
:100B3000206578292050696E67204E554D20494424
:100B40002064796E616D6978656C2E000D0A205302
:100B50005752205B414444525D5B4C454E5D5B49BE
:100B6000445D5B444154415D2E2E2E5B49445D5BE8
:100B7000444154415D2E2E2E203A2053796E63203D
:100B800057726974652E000D0A205343414E205B55
:100B90004E554D5D203A205343414E206C696E6B9B
:100BA00065642064796E616D6978656C20696E207A
:100BB000307E4E554D20696E2063757272656E747D
:100BC000206261756420726174652E000D0A204CEC
:100BD0004544205B4E554D5D203A20426C696E6B5A
:100BE000204C4544206F66204E554D2049442E2010
:100BF0002742272C274E2720666F72204944206306
:100C000068616E67652E2027512720666F7220511C
:100C10007569742E000D0A2042415544205B4E55E3
:100C20004D5D203A205365742062617564207261C5
:100C300074652020657829204241554420323228AD
:100C40003537363030425053292C2042415544200C
:100C50003128314D42505329000D0A20534541524D
:100C60004348203A205365617263682049442061FB
:100C70006E64206261756472617465206F662061C4
:100C80006C6C206C696E6B65642064796E616D6953
:100C900078656C732E000D0A2055706461746520B0
:100CA0005B53544152545F49445D205B454E445F61
:100CB00049445D203A2044796E616D6978656C2005
:100CC0006669726D77617265207570646174652EF6
:100CD0002873797374656D2075736572206F6E6CFF
:100CE0007929000D0A0A2020202020202020436F8F
:100CF0007079726967687420524F424F544953208B
:100D0000434F2E2C4C54442E0D0A005B496E7661E5
:100D10006C6964205061676520526561643A000D1A
:100D20000A205B4572723A5278442054696D656FAF
:100D300075745D000D0A205B4572723A57726F6ED2
:100D400067204865616465725D000D0A205B45722D
:100D5000723A5478494420213D20527849445D003C
:100D60000D0A205B4572723A57726F6E67204C65B0
:100D70006E6774685D000D0A205B4572723A5772A7
:100D80006F6E6720436865636B53756D5D000D0A78
:100D900020555044415445205B53544152542049FE
:100DA000445D205B454E442049445D005D3A000DA2
:100DB0000A2049443A00205374616E6462792E001F
:100DC0002057726974696E672E2E00205375636315
:100DD0006573732E00204572726F722E000D0A200B
:100DE0004572722049443A002042616420436F6D8D
:100DF0006D616E64005B457869745D005B53544FB0
:100E0000505D000D0A204D4F54494F4E20504C412B
:100E10005920504147452020202028522F57290093
:100E20000D0A204F4E20504C4159494E47204D4FFE
:100E300054494F4E2020202028522920000D0A20FE
:100E4000545820574952454C455353205041434B29
:100E50004554202028522F5729000D0A205258208F
:100E6000574952454C455353205041434B4554201C
:100E7000202028522920000D0A204E45572050419D
:100E8000434B455420415252495645442020202886
:100E9000522920000D0A20415558204C454420205D
:100EA000202020202020202020202028522F5729B9
:100EB000000D0A20425554544F4E282D532D552DC8
:100EC000442D4C2D522920202028522920000D0A83
:100ED0002054494D4552283132356D5365632045C4
:100EE000616368292028522F5729000D0A205A498A
:100EF0004742454520494420202020202020202012
:100F0000202028522F5729000D0A20524F424F54BB
:100F1000204944202020202020202020202020287C
:100F2000522F5729000D44796E616D6978656C20E8
:100F300020302830783030295B202020205D000DC3
:100F40000A44796E616D6978656C202031283078AB
:100F50003031295B202020205D0020506167654EE4
:100F6000756D6265723A000D0A44796E616D69783B
:100F7000656C2020322830783032295B20202020F8
:100F80005D0020416464723A000D0A44796E616D1F
:100F90006978656C2020332830783033295B202035
:100FA00020205D00202852657365727665642920D3
:100FB0003A000D0A44796E616D6978656C202034C1
:100FC0002830783034295B202020205D002020202C
:100FD000506C6179436F756E743A000D0A44796EF6
:100FE000616D6978656C2020352830783035295B53
:100FF000202020205D00202852657365727665648C
:1010000029203A000D0A44796E616D6978656C207B
:1010100020362830783036295B202020205D0020C3
:1010200028526573657276656429203A000D0A447A
:10103000796E616D6978656C20203728307830379B
:10104000295B202020205D00202852657365727680
:10105000656429203A000D0A44796E616D697865EE
:101060006C2020382830783038295B202020205D03
:10107000002028526573657276656429203A000D58
:101080000A44796E616D6978656C20203928307862
:101090003039295B202020205D002020205061670E
:1010A0006520537465703A000D0A44796E616D696C
:1010B00078656C2031302830783041295B20202041
:1010C000205D0020436F6E74726F6C436F64653AED
:1010D000000D0A44796E616D6978656C20313128A4
:1010E00030783042295B202020205D002020506194
:1010F00067652053706565643A000D0A44796E6136
:101100006D6978656C2031322830783043295B2056
:101110002020205D0020202044584C205365747509
:10112000703A000D0A44796E616D6978656C203102
:10113000332830783044295B202020205D00202097
:10114000416363656C2054696D653A000D0A44790A
:101150006E616D6978656C203134283078304529AE
:101160005B202020205D004C696E6B20746F204E48
:101170006578743A000D0A44796E616D6978656C22
:101180002031352830783046295B202020205D0032
:101190004C696E6B20746F20457869743A000D0AB3
:1011A00044796E616D6978656C203136283078310C
:1011B00030295B202020205D0028526573657276FF
:1011C00065645031293A000D0A44796E616D697881
:1011D000656C2031372830783131295B2020202080
:1011E0005D002852657365727665645231293A0054
:1011F0000D0A44796E616D6978656C20313828304C
:10120000783132295B202020205D002852657365EB
:10121000727665645032293A000D0A44796E616D28
:101220006978656C2031392830783133295B20208A
:1012300020205D00285265736572766564523229FC
:101240003A000D0A44796E616D6978656C20323020
:101250002830783134295B202020205D000D0A449D
:10126000796E616D6978656C20323128307831355E
:10127000295B202020205D000D0A44796E616D6994
:1012800078656C2032322830783136295B20202076
:10129000205D000D0A44796E616D6978656C2032BD
:1012A000332830783137295B202020205D000D0A5B
:1012B00044796E616D6978656C20323428307831FC
:1012C00038295B202020205D000D0A44796E616D75
:1012D0006978656C2032352830783139295B2020D7
:1012E00020205D000D0A44796E616D6978656C207F
:1012F00032362830783161295B202020205D000DB6
:101300000A44796E616D6978656C203237283078CF
:101310003162295B202020205D000D0A44796E6136
:101320006D6978656C2032382830783163295B200C
:101330002020205D000D0A44796E616D6978656C2E
:101340002032392830783164295B202020205D004C
:101350000D0A44796E616D6978656C2033302830F0
:10136000783165295B202020205D000D0A20202097
:10137000506175736554696D652020202020202000
:101380005B2020205D000D0A2020205370656564DD
:1013900020202020202020202020205B2020205DD5
:1013A000202020202020202020202020202020203D
:1013B000202020202020202020202020202020202D
:1013C000202020205B583A2D2D2C593A2D2D2C41D0
:1013D0003A2D2D2D2D5D000D0A20202020202020CB
:1013E000202020202020202020202020535450374F
:1013F00020205354503020535450312053545032F5
:1014000020535450332053545034205354503520DB
:101410005354503620202020476F20537465703A73
:101420002020202020000D0A202020202020202005
:1014300020202020202020202020202020202020AC
:10144000204D53545220534C4156204F4653542064
:10145000202020202020202020202020202020208C
:1014600020202020202020476F20537465703A20D0
:1014700020202020000D0A5D205F20202020202039
:10148000202020202020202020202020202020205C
:10149000202020202020202020202020202020204C
:1014A000202020202020202020202020202020203C
:1014B000202020202020202020202020202020202C
:1014C000202020002041726520796F75207375728D
:1014D000653F5B792F4E5D0020496E76616C6964D3
:1014E00020506167650020496E76616C6964205008
:1014F0006172616D6574657200204F666673657414
:10150000205570646174656400204F7574206F66A7
:101510002052616E676500204F4B000D0A2020208D
:1015200020202020202D434D3A2052503D2850614C
:101530007261302C4F502C506172613129204C4B1C
:10154000205253205B414444525D2020000D0A206C
:10155000427265616B20617420000D0A2045525271
:101560004F523A004946202020202000454C534548
:1015700020494600454C534520202000616E642FD1
:101580006F7220004A554D50202020004C4F41449E
:1015900020202000434F4D50555445005354415294
:1015A00054202000454E44202020200043414C4C34
:1015B0002020200052455455524E20004E554C4C90
:1015C000202020000D0A204845584120444953500E
:1015D0004C4159204D4F4445000D0A204445434994
:1015E0004D414C20444953504C4159204D4F4445A6
:1015F0000003404C464D4840454A230102030A225D
:101600002121217D7D7D7D7D7D7D7D7D7D7D7D7D1E
:101610007D7D797673716E6C6967656361605E5C10
:101620005B59585755545351504F4E4D4C4B4A49A6
:10163000484746454443424241403F3F3E3D3C3C93
:101640003B3A39393837373636353434333332313B
:101650003130302F2F2E2D2D2C2C2B2B2A2A2929BF
:10166000282827272626252525242423232222212E
:10167000212020201F1F1E1E1D1D1D1C1C1B1B1A90
:101680001A1A1919181818171716161615151414EA
:1016900014131312121211111010100F0F0E0E0E40
:1016A0000D0D0C0C0C0B0B0A0A0909090808070799
:1016B00007060605050404040303020201010100F4
:1016C000000000000000000000000000000000001A
:1016D000000000000000000000000000000000000A
:1016E00000000000000000000000000000000000FA
:1016F00000000000000000000000000000000000EA
:1017000000000000000001010102000200010101CF
:1017100001020001010101020002000101010101B9
:1017200001020002000200020002000200010101A9
:10173000010101020001010200020000000001019C
:10174000010101000001010101010001010101018C
:101750000100000101000000000000010000000184
:10176000010200010100000101010102000200016B
:011770000177
:10177200682FA901812F0023B9F40FE003BF00E015
:1017820002BF09E01DE30E94704D10E0003021E02D
:10179200120710F000E009C001BF082F00FB07B7D5
:1017A20001F907BF01E001C000E0862F089500E0C3
:1017B2000093610002B901BB04BB07BB0ABB00E096
:1017C200009365000093620003B902BB05BB08BB2E
:1017D20000B50B7F00BD00B50B7F00BD00E000939C
:1017E200610002B901BB04BB07BB0ABB00E0009366
:1017F20065000093620003B902BB05BB08BBBD9A3A
:10180200C59A909A1C9A1D9A1E9A1F9A04B30F6742
:1018120004BB02B10C6002B9AC9AAB9AAA9AA99A1B
:10182200A89AAE9AAD9AAC9AAB9AAA9AA99AA89A91
:101832001A981B9A01B3006701BB9798949A959ADC
:101842009698AC9AAB9AAA9AA99AA89A0895002354
:1018520091F400E00093900019B902E00BB908E19D
:101862000AB920FB0EF4579A06E0009395000FEF99
:101872000CB95E9A08950130E9F400E000939800F3
:101882001093990002E000939B0008E100939A00F4
:1018920020FB2EF400919A00006800939A0006E063
:1018A20000939D000FEF00939C0000919B00006449
:1018B20000939B000895592F482F80E090E008C0C4
:1018C2002FE93FE021503040E9F700C000000196C7
:1018D20080179107A8F3842F952F08959A938A93DE
:1018E20080E090E088D20A3318F00753102F02C02C
:1018F2000053102F012F10E0102F00E0110F110FD5
:10190200110F110F802B912B76D20A3318F0075347
:10191200102F02C00053102F012F302F20E0822BF6
:10192200932B69D20A3318F00753102F02C00053C9
:10193200102F012F10E044E00E94644D802B912B68
:101942005AD20A3318F00753102F02C00053102F37
:10195200012F10E0802B912B8C0189919991089590
:101962000E94064E229728833983B02FD12E7A0106
:1019720082E090E001E00093E80CBB249699B394D6
:10198200CC249599C394969A959825C0949801E091
:1019920010E091DF00E00093FE0C0093FD0C949A9E
:1019A20005E010E088DF01E2F5D001E311E083DF1A
:1019B20008E0F0D00091FD0C1091FE0C011751F0DF
:1019C2000091FD0C1091FE0C011721F014D201328E
:1019D200B9F791E08A95813010F09923B9F29923F1
:1019E20009F4A1C000E00093FE0C0093FD0C442416
:1019F200552466247724A0E08824992409E6CAD0D5
:101A020008E0C8D0F8D10A33E9F7F5D10A33E9F78B
:101A120065DF2801F0D10A33E9F760DF38010FEF03
:101A220060160FEF700649F0E6D10A33E9F7E3D109
:101A3200093511F4A1E001C0A0E00EE110E03BDFA6
:101A420000E00093FE0C0093FD0C02E5A3D008E039
:101A5200A1D0D1D1802F8C3641F4CDD10A33E9F710
:101A62003DDF4801AA24A39403C08F3691F7AA242C
:101A7200E2EEFCE040825182E4EEFCE060827182A0
:101A8200E6EEFCE080829182B0FBC6F404E110E055
:101A920012DF04E47FD008E07DD0ADD10A33E9F74C
:101AA20005E010E008DF088119817BD108E072D0DF
:101AB20008E070D008E06ED008E06CD0B1FB4EF4C4
:101AC20004E110E0F8DEDA1621F007E563D008E061
:101AD20061D0B2FBCEF4AA20B9F004E110E0EBDE53
:101AE20003E458D008E056D086D10A33E9F705E07E
:101AF20010E0E1DE870155D108E04CD008E04AD081
:101B020008E048D008E046D004E110E0D4DE05E465
:101B120041D008E03FD0949801E010E0CCDE949AE6
:101B220004E610E0C8DE00E00093FE0C0093FD0C1A
:101B32000B2D00FD969A00FF96980C2D00FD959AAC
:101B420000FF959800E00093E80C092F2296E0E14F
:101B52000C94174E5E9A1B981A9A18D05E9BFECF71
:101B62001A981B9A08958A93802F082F02950F7056
:101B7200005D0A3308F0095F0DD08F70805D082F79
:101B82000A3308F0095F06D0899108955D9BFECF64
:101B92000CB90895A99810919B00212F25FFFBCF26
:101BA20000939C0008959A938A93802F082F44E60D
:101BB2000E94464D902F092F005DECDF04E6909FB6
:101BC2008019082F4AE00E94464D902F092F005D90
:101BD200E1DF0AE0909F8019805D082FDBDF8991A9
:101BE200999108950E94084E48015901DD24BB20B5
:101BF20052F49094A094B094000B8194900AA00A9D
:101C0200B00A0DE2C7DF80E09AECAAE9BBE3CC247C
:101C12001AC0DD2019F08201005DBCDF8201930150
:101C2200AC01BD010E94954D801A910AA20AB30A25
:101C32008C019D014AE050E060E070E00E94DF4DBF
:101C4200C801D901C39409E0C016A8F48401950122
:101C5200AC01BD010E94DF4D402E5524662477243D
:101C6200042D052906290729A1F28201005D92DFD0
:101C7200DD24D394D3CF84019501AC01BD010E9430
:101C8200DF4D402E552466247724042D005D82DF2B
:101C9200EEE00C94194E0E940E4E38015524A0E13C
:101CA200B7E244240FC000E375DF8C01AD010E944E
:101CB200544D601A710A8D014AE050E00E94704D45
:101CC200D801439405E04016D0F48301AD010E948F
:101CD200704DC801082F092B31F0082F005D5ADF23
:101CE20055245394E2CF552021F0082F005D52DF96
:101CF200DCCF04E04016B8F600E24CDFD6CFE8E0D5
:101D02000C941F4E10915F09112311F02CDF0895DE
:101D120023E010E00AD0089520915F09222311F0F8
:101D220040D0089524E001D008950E940C4E38015D
:101D3200822E5524A0E1B7E244240FC000E32ADF3B
:101D42008C01AD010E94544D601A710A8D014AE066
:101D520050E00E94704DD801439405E04016F0F423
:101D62008301AD010E94704DC80104E010E0242DF2
:101D720030E0021B130B9924081519050CF7082FE4
:101D8200092B31F0082F005D05DF55245394D8CF7D
:101D92005520A1F2082F005DFDDED2CFEAE00C94BF
:101DA2001D4E9A938A93C8018C01012F10E0DBDE4D
:101DB200082FD9DE8991999108950E94124EC80187
:101DC200D9018C019D01022F132F330F220B330BEC
:101DD200E8DF8C01E6DFE4E00C94234EBA93AA9389
:101DE200D80103C00C91D6DE11960C910023D1F7D5
:101DF200A991B99108950091FE0C1091FD0C011763
:101E0200D1F30091FE0C102F13951093FE0C10E0ED
:101E12000F701070F801E150F34F008108958A931A
:101E2200802F082FC0DE08E2B5DE00E3B3DE08E54E
:101E3200B1DE082F98DE09E2ADDE899108950E9495
:101E42000B4EEF97EF97EF972797A898992401E009
:101E52000093680901E00093670905C004E110E0FE
:101E62002ADD08E001BD992011F00C948C1706EAD6
:101E720015E0B4DF00915809D2DF0FEA15E0AEDFBA
:101E820020E08E0108571F4F0E943D1F00E008838B
:101E9200AE0148575F4F9E01205F3F4F8E010E9467
:101EA200911D802E00916509009366098820D9F260
:101EB2000FE1801610F00EE1802E2AE536E08E0149
:101EC2000E946F1D002351F628E536E08E010E9424
:101ED2006F1D002309F450C007EB10E00E94444B31
:101EE20080E01CC0FE017096082F10E0000F111F49
:101EF200000F111FE00FF11F008111812281338138
:101F020090E0FC01E553F74F008390E0FC01E553BC
:101F1200F74F0081F7DE00E23DDE839590E0E82D89
:101F2200F0E031978E179F07ECF21B981A9A80E027
:101F320008C090E0FC01E553F74F008127DE5E9A6E
:101F4200839590E0E82DF0E031978E179F078CF390
:101F52005E9BFECF1A981B9A0FEF0E94E9480093EE
:101F6200690909EC10E00E94444B2091690907E1DC
:101F720018E00E94F64977CF23E536E08E010E94F1
:101F82006F1D002371F420E536E08E010E946F1D63
:101F9200002339F42EE436E08E010E946F1D0023E7
:101FA20069F100915809083CB1F40CE810E00E9474
:101FB200444B088919892A893B8931DF0AE3EADD22
:101FC200088919892A893B89102F009158090E9492
:101FD200DC3BA2DE48CF088919892A893B89009314
:101FE20095070C891D892E893F890093960722E067
:101FF20012E0009158090E94204A35CF21EA35E0CB
:102002008E010E946F1D0023A9F014E3009158096C
:102012000E94ED4CC801282F14E1009158090E943A
:10202200091D892F90E0282F15E1009158090E947F
:10203200091D19CF2CE935E08E010E946F1D002386
:1020420031F114E3009158090E94ED4CD80114E1DA
:10205200009158090E94ED4CC80116E100915809FF
:102062000E94ED4C080F191F169507950A1B1B0BB2
:10207200212F27FF04C00195006810E001C010E085
:10208200202F1AE0009158090E94091DECCE28E980
:1020920035E08E010E946F1D002341F001E00093A4
:1020A2005F0904EC15E10E94444BDDCE24E935E0E2
:1020B2008E010E946F1D002341F000E000935F0932
:1020C20009ED15E10E94444BCECE2FE835E08E019A
:1020D2000E946F1D0023A9F014E3009158090E9489
:1020E200ED4CC801282F16E1009158090E94091DE4
:1020F200892F90E0282F17E1009158090E94091DAD
:10210200B2CE2BE835E08E010E946F1D002339F418
:1021120023E835E08E010E946F1D0023F9F080E074
:1021220014C0FE017096082F10E0000F111F000F5F
:10213200111FE00FF11F008111812281338190E094
:10214200FC01EB56F84F00838395881550F38A946F
:10215200282D13E80EEF0E94204A85CE2DE735E0A8
:102162008E010E946F1D002371F42AE735E08E0173
:102172000E946F1D002339F428E735E08E010E948A
:102182006F1D0023A1F100915809083C81F40C89CC
:102192001D892E893F899801488959896A897B89D5
:1021A2008A01102F009158090E94C93A5CCE80E042
:1021B20014C0FE017096082F10E0000F111F000FCF
:1021C200111FE00FF11F008111812281338190E004
:1021D200FC01EB56F84F00838395881550F38A94DF
:1021E200282D13E0009158090E94204A3CCE21E795
:1021F20035E08E010E946F1D002301F180E014C0C2
:10220200FE017096082F10E0000F111F000F111F22
:10221200E00FF11F008111812281338190E0FC01E6
:10222200EB56F84F00838395881550F38A94282D36
:1022320014E0009158090E94204A15CE2AE635E0A2
:102242008E010E946F1D002339F426E635E08E01CF
:102252000E946F1D0023F9F080E014C0FE01709609
:10226200082F10E0000F111F000F111FE00FF11FC8
:10227200008111812281338190E0FC01EB56F84FFD
:1022820000838395881550F38A94282D15E00EEF6C
:102292000E94204AE8CD2FE535E08E010E946F1D95
:1022A200002381F00C891D892E893F89202F4889BE
:1022B20059896A897B898A01102F009158090E94E5
:1022C200091DD1CD29E535E08E010E946F1D002345
:1022D20021F104EF10E00E94444B8DDD093719F023
:1022E200093509F0C0CD01E0801619F400915809B2
:1022F20004C0088919892A893B8920E016E00E94D6
:10230200204A002309F4AFCD01E00093580921E0EF
:1023120030E0A9010E94424DA6CD22E535E08E01B2
:102322000E946F1D0023A1F001E0801639F420E025
:1023320017E0009158090E94204A95CD20E017E04D
:10234200488959896A897B89042F0E94204A8BCD4A
:102352002FE435E08E010E946F1D002339F42DE435
:1023620035E08E010E946F1D0023D9F102E0801634
:1023720019F003E0801681F50EE1009395070889B4
:1023820019892A893B8900939607088919892A891C
:102392003B89012F10E00093970703E08016A9F410
:1023A2000C891D892E893F89009398070C891D8904
:1023B2002E893F89012F10E00093990725E013E051
:1023C200009158090E94204A4ECD23E013E000916B
:1023D20058090E94204A47CD0BE011E00E94444B6D
:1023E20042CD28E435E08E010E946F1D002379F072
:1023F20001E0801619F40091580904C0088919896E
:102402002A893B8920E011E00E94204A2CCD25E454
:1024120035E08E010E946F1D002349F103E0009315
:102422009507088919892A893B890093960706E34B
:1024320011E00E94444B0091960764DC0CE511E028
:102442000E94444BD8DC093519F0093709F00BCD4D
:1024520022E013E00EEF0E94204A009196070093BB
:10246200580921E030E0A9010E94424DFCCC20E451
:1024720035E08E010E946F1D002339F42BE036E017
:102482008E010E946F1D0023E1F000915809083C63
:1024920011F494D5E8CC00E0009395070AE3009389
:1024A200960722E012E0009158090E94204A002378
:1024B20009F4D9CC009158090E3F09F4D4CC7ED549
:1024C200D2CC24E036E08E010E946F1D002309F475
:1024D2003FC103E0801651F4488859886A887B8896
:1024E2000C891D892E893F89A02E0DC002E080161D
:1024F20031F4488859886A887B88A42C04C00EE885
:102502001DE00E94444B02E0801621F003E0801699
:1025120009F0A9CC00E0009367090093680909B1AA
:10252200023289F421E014E00EEF0E94034D0AE02A
:1025320010E0C1D901E009B90093570920E030E069
:10254200A9010E94424D22E214E00EEF0E94034DC7
:102552000AE010E0B0D902E209B90093570920E07D
:1025620030E0A9010E94424D00E00E945F4B05C08D
:1025720001E711E00E94444B4394A41408F4DAC02A
:102582005524F201E659F64F00810023A9F30FEA20
:102592001DE00E94444B042DB5DB90E0992399F491
:1025A20091E080E08F31D0F7082F0E94411D002377
:1025B20041F020E011E0082F0E94204A002309F494
:1025C20090E08395EFCF06EB1DE00E94444B80E044
:1025D2000FC0841561F090E0FC01E659F64F0081CE
:1025E200002329F025E01DE2082F0E94091D839592
:1025F2008F3178F300EC1DE00E94444B2FEF1AEF6D
:10260200042D0E94091D2EEF1DE2042D0E94091DBA
:10261200002309F4ADCF04E610E04DD90DE09ADABB
:1026220000E00E94C31C0CE495DA00E00E94C31C87
:102632001B981A9A80E090ECA0E0B0E05524662442
:10264200772412C0FC013A2F3BBF069000E00BBF7B
:102652008F5F9F4FAF4FBF4F500C002D97DA5E9A9E
:1026620001E0600E00E0701E0FEF601607E17006D9
:1026720048F3052D8BDA5E9A5E9BFECF1A981B9A61
:1026820000E00E94C31C06E565DA00E00E94C31C5C
:1026920000E001C00395043638F410E0F801E95E69
:1026A200F74F10811D32B1F70395202F01C003951A
:1026B200043638F410E0F801E95EF74F10811D325C
:1026C200B1F7039510E001C01395183090F4602F14
:1026D200062F0395422F242F239570E0FB01E95E1C
:1026E200F74F308150E0FA01E95EF74F408134172D
:1026F20059F31830D1F40BEC1DE00E94444B01E475
:1027020029DA00E00E94C31C07E424DA00E00E94F8
:10271200C31C20E017E0042D0E94204A0CE211E0C5
:10272200CAD800E00093670927CF05ED1DE00E949B
:10273200444B22CF0E940D4B09B10093570920E070
:1027420030E0A9010E94424D01E0009368098BCB61
:102752002FEF35E08E010E946F1D002309F440C067
:10276200B091670900E0009368090093670980E06F
:1027720001E0801611F4AEEF05C0088919892A8993
:102782003B89A02F0CE810E00E94444B90E005C06A
:102792000DE200DA0DE5FED993959A1788F40BE560
:1027A200F9D9092FAFDA0AE3F5D920E011E0092FB0
:1027B2000E94204A002361F30FE4ECD98395EACF0B
:1027C2000CE810E00E94444B082F29DB08E512E0D8
:1027D2000E94444BB093670901E00093680943CB20
:1027E2002BEF35E08E010E946F1D002309F44EC0CD
:1027F20001E0801619F4A091580905C008891989C9
:102802002A893B89A02F01E00093670900E0009329
:10281200680903EA11E00E94444B80E007E412E0F9
:102822000E94444B0A2F6EDA0091FE0C1091FD0CAF
:10283200011791F0E0DA802F823411F0823609F428
:10284200AA958E3411F08E3609F4A3950BE612E0A8
:102852000E94444B0A2F56DA21E019E10A2F0E9406
:10286200034D04E610E027D820E019E10A2F0E9468
:10287200034D04E610E01FD8813521F0813711F0B5
:102882008B3191F601E000936809EDCA24EF35E03F
:102892008E010E946F1D002309F48EC000E0009398
:1028A20068090AE077D980E001C083958E3F08F07D
:1028B20078C089B920E011E00EEF0E94204A0DE0B5
:1028C20069D980FB1EF40BE265D902C00AE262D923
:1028D20000916909002309F45DC0A0E056C0B0E090
:1028E200FD01E95EF74F00810F3F09F04DC00A2F4D
:1028F20010E00F5F1F4FF801E95EF74F00810F3FB5
:1029020009F042C00A2F10E00D5F1F4FF801E95E87
:10291200F74F00810230C1F50A2F10E00E5F1F4F02
:10292200F801E95EF74F408150E00A2F10E00D5F99
:102932001F4FF801E95EF74F208130E0240F351F69
:102942000A2F10E00B5F1F4FF801E95EF74F00817D
:1029520010E0020F131F0F3F20E01207A9F40CE74B
:1029620012E00E94444B082FCDD90FE812E00E94DA
:10297200444B0A2F10E00E5F1F4FF801E95EF74F3C
:102982000081C0D90AE006D9A39500916909A01770
:1029920008F4A5CF0091FE0C1091FD0C011709F46B
:1029A20084CF0091570909B901E0009368090DE04D
:1029B200F1D800E2EFD857CA2FEE35E08E010E941F
:1029C2006F1D002391F104E000939507088919898E
:1029D2002A893B890093960722E013E00EEF0E94BA
:1029E200204A05E912E00E94444B00E814E82EE177
:1029F20030E0488959896A897B894F5F5F4F6F4F01
:102A02007F4F0E94B94DEED800EB12E00E94444B7A
:102A1200088919892A893B8909B90093570920E055
:102A220030E0A9010E94424D1ECA27EE35E08E0118
:102A32000E946F1D002309F442C001E0801631F4A8
:102A420000E1402E55246624772404C04888598822
:102A52006A887B8800EC11E00E94444B2BC00091F5
:102A62006609109165090117A1F080E090E0A0E0ED
:102A7200B0E0AA240091660910E0F801EB56F94F84
:102A82000081E6E6F9E01081139510833BD900E25C
:102A920081D88F5F9F4FAF4FBF4F84159505A60515
:102AA200B705E8F2AA2031F40DE074D80AE072D832
:102AB200AA24A39480E090E0A0E0B0E0EECF22EE62
:102AC20035E08E010E946F1D002309F44AC0488838
:102AD20059886A887B888C899D89AE89BF8904EB75
:102AE20012E00E94444B042D0DD90FEB12E00E941C
:102AF200444B8C0111D909EC12E00E94444BA0E036
:102B020006C021E018E10A2F0E94034DA3954A1640
:102B1200C0F70AED12E00E94444B0CC02FEF33E0E5
:102B22001EE10A2F0E940B4DA3954A16B8F78C019D
:102B32000E945C0C0091FE0C1091FD0C011709F033
:102B420092C9A0E007C020E030E01EE10A2F0E94F7
:102B52000B4DA3954A16B8F78C010E945C0CA0E0BD
:102B6200E4CF2EED35E08E01B9D7002309F431C14F
:102B720000E000936809009158090093950721E04D
:102B820015E00EEF0E94204A01E0801641F520E197
:102B920030E0A9010E94364D802E80E090E0E82DC1
:102BA200F0E031978E179F070CF042C0E82FF0E05B
:102BB2007196AF010E94364D10E020E030E0FE0138
:102BC2007096482F50E0440F551F440F551FE40FD5
:102BD200F51F00831183228333838395DFCF05E1C1
:102BE200801610F004E1802E20E130E0082DA901CA
:102BF2000E94424D80E015C0FE017096082F10E041
:102C0200000F111F000F111FE00FF11F0081118132
:102C120022813381E82FF0E07196AF010E94424D8C
:102C2200839590E0E82DF0E031978E179F0724F30B
:102C32000CE810E00E94444B0BE50E94CB0D80E0B3
:102C420004C00DE50E94CB0D839590E0E82DF0E0E5
:102C520031978E179F07D4F4FE017096082F10E06B
:102C6200000F111F000F111FE00FF11F00811181D2
:102C72002281338147D890E0E82DF0E032978E1719
:102C82009F07FCF60DE20E94CB0DDECF0091FE0CF9
:102C92001091FD0C011709F098C00CE810E00E9499
:102CA200444B80E018C0FE017096082F10E0000F20
:102CB200111F000F111FE00FF11F008111812281EE
:102CC2003381102F009158090E94DE4C1BD800E27C
:102CD2000E94CB0D839590E0E82DF0E031978E179E
:102CE2009F07A4F6FE017096082F10E0000F111F37
:102CF200000F111FE00FF11F00811181228133812A
:102D0200083CF9F000915809043688F100915809FD
:102D12000E3668F50BE317E1FE017096282F30E0BE
:102D2200220F331F220F331FE20FF31F4081518105
:102D32006281738150E0040F151FF8010491023083
:102D4200B1F4FE017096082F10E0000F111F000F62
:102D5200111FE00FF11F0081118122813381102F99
:102D6200009158090E94DC3B0E948D0EB0CF03E017
:102D720017E1FE017096282F30E0220F331F220F39
:102D8200331FE20FF31F408151816281738150E052
:102D9200040F151FF8010491023009F084CFFE01DF
:102DA2007096082F10E0000F111F000F111FE00F87
:102DB200F11F0081118122813381102F0091580966
:102DC2000E94ED4C0E948D0E82CF01E000936809B3
:102DD2004AC829ED35E08E0181D6002389F1488861
:102DE20059886A887B888C899D89AE89BF8900E071
:102DF20000936809A0E04A1698F021E018E10A2F32
:102E02000E94034DA395F7CF2FEF33E01EE10A2F67
:102E12000E940B4DA3954A16B8F78C010E945C0CD8
:102E2200A0E007C020E030E01EE10A2F0E940B4D17
:102E3200A3954A16B8F78C010E945C0CA0E0EBCF78
:102E420025ED35E08E014AD6002361F00889198903
:102E52002A893B890093580921E030E0A9010E94A8
:102E6200424D01C820ED35E08E0138D6002331F401
:102E72002EEC35E08E0132D6002321F00E945A4812
:102E82000C94340F28EC35E08E0128D6002331F45F
:102E920026EC35E08E0122D6002321F00E948D48D7
:102EA2000C94340F21EC35E08E0118D6002319F072
:102EB2003CD00C94340F2DEB35E08E010FD600235D
:102EC20081F002E0801640F0088919892A893B893D
:102ED2000E9497400C94340F01E00E9497400C949A
:102EE200340F26EB35E08E01F9D5002331F422EBC5
:102EF20035E08E01F3D5002321F0992493940C94AC
:102F0200340F0CE810E00E94444B08EE1DE00E94D2
:102F1200444B0C94340F00E000936809EF96EF964F
:102F2200EF962796EBE00C941C4E03E319E00E9407
:102F3200444B05E519E00E94444B0BE719E00E945F
:102F4200444B00EA19E00E94444B09EE19E00E944A
:102F5200444B00E31AE00E94444B07E61AE00E9449
:102F6200444B0DE81AE00E94444B08EC1AE00E9420
:102F7200444B06E01BE00E94444B02E21BE00E942D
:102F8200444B0CE41BE00E94444B07E81BE00E9408
:102F9200444B0CEC1BE00E94444B05E11CE00E94F8
:102FA200444B09E51CE00E94444B06E91CE00E94E8
:102FB200444B03EE1CE00E94444B08950E94124EC3
:102FC20000915809083C09F0B9C088E103E01EE00D
:102FD2000E94444B082F0E94100F0AE30E94CB0D5F
:102FE200182F009158090E94DC3B0E948D0E839598
:102FF20000E21EE00E94444B082F0E94100F0AE3D9
:103002000E94CB0D182F009158090E94DC3B0E94B0
:103012008D0E83950DE31EE00E94444B082F0E9403
:10302200100F0AE30E94CB0D182F009158090E943D
:10303200DC3B0E948D0E839583950AE51EE00E947B
:10304200444B082F0E94100F0AE30E94CB0D182F49
:10305200009158090E94DC3B0E948D0E8395839556
:1030620007E71EE00E94444B082F0E94100F0AE35C
:103072000E94CB0D182F009158090E94DC3B0E9440
:103082008D0E839504E91EE00E94444B082F0E9496
:10309200100F0AE30E94CB0D182F009158090E94CD
:1030A200DC3B0E948D0E839501EB1EE00E94444B97
:1030B200082F0E94100F0AE30E94CB0D182F0091D7
:1030C20058090E94DC3B0E948D0E83950EEC1EE097
:1030D2000E94444B082F0E94100F0AE30E94CB0D5E
:1030E200182F009158090E94DC3B0E948D0E839597
:1030F2000BEE1EE00E94444B082F0E94100F0AE3C1
:103102000E94CB0D182F009158090E94DC3B0E94AF
:103112008D0E8395839508E01FE00E94444B082F93
:103122000E94100F0AE30E94CB0D182F009158093C
:103132000E94DC3B0E948D0E839521C480E008E052
:1031420013E00E94444B082F0E94100F0CEA1DE06E
:103152000E94444BA82FB0E01596FD01E95EF74F9F
:1031620000810E94100F839507E313E00E94444BF5
:10317200082F0E94100F0CEA1DE00E94444BA82F5A
:10318200B0E01596FD01E95EF74F00810E94100F35
:10319200839506E513E00E94444B082F0E94100F0E
:1031A2000CEA1DE00E94444BA82FB0E01596FD01E9
:1031B200E95EF74F00810E94100F839505E713E047
:1031C2000E94444B082F0E94100F0CEA1DE00E943F
:1031D200444BA82FB0E01596FD01E95EF74F008140
:1031E2000E94100F839504E913E00E94444B082FBC
:1031F2000E94100F0CEA1DE00E94444BA82FB0E081
:103202001596FD01E95EF74F00810E94100F83952C
:1032120003EB13E00E94444B082F0E94100F0CEAAC
:103222001DE00E94444BA82FB0E01596FD01E95E17
:10323200F74F00810E94100F839502ED13E00E9468
:10324200444B082F0E94100F0CEA1DE00E94444BD1
:10325200A82FB0E01596FD01E95EF74F00810E94AC
:10326200100F839501EF13E00E94444B082F0E9438
:10327200100F0CEA1DE00E94444BA82FB0E01596F7
:10328200FD01E95EF74F00810E94100F839500E176
:1032920014E00E94444B082F0E94100F0CEA1DE01C
:1032A2000E94444BA82FB0E01596FD01E95EF74F4E
:1032B20000810E94100F83950FE214E00E94444B9C
:1032C200082F0E94100F0CEA1DE00E94444BA82F09
:1032D200B0E01596FD01E95EF74F00810E94100FE4
:1032E20083950EE414E00E94444B082F0E94100FB5
:1032F2000CEA1DE00E94444BA82FB0E01596FD0198
:10330200E95EF74F00810E94100F83950DE614E0ED
:103312000E94444B082F0E94100F0CEA1DE00E94ED
:10332200444BA82FB0E01596FD01E95EF74F0081EE
:103332000E94100F83950CE814E00E94444B082F62
:103342000E94100F0CEA1DE00E94444BA82FB0E02F
:103352001596FD01E95EF74F00810E94100F8395DB
:103362000BEA14E00E94444B082F0E94100F0CEA53
:103372001DE00E94444BA82FB0E01596FD01E95EC6
:10338200F74F00810E94100F83950AEC14E00E940F
:10339200444B082F0E94100F0CEA1DE00E94444B80
:1033A200A82FB0E01596FD01E95EF74F00810E945B
:1033B200100F839509EE14E00E94444B082F0E94DF
:1033C200100F0CEA1DE00E94444BA82FB0E01596A6
:1033D200FD01E95EF74F00810E94100F839508E01E
:1033E20015E00E94444B082F0E94100F0CEA1DE0CA
:1033F2000E94444BA82FB0E01596FD01E95EF74FFD
:1034020000810E94100F839507E215E00E94444B51
:10341200082F0E94100F0CEA1DE00E94444BA82FB7
:10342200B0E01596FD01E95EF74F00810E94100F92
:10343200839506E415E00E94444B082F0E94100F6A
:103442000CEA1DE00E94444BA82FB0E01596FD0146
:10345200E95EF74F00810E94100F839505E615E0A3
:103462000E94444B082F0E94100F0CEA1DE00E949C
:10347200444BA82FB0E01596FD01E95EF74F00819D
:103482000E94100F839504E815E00E94444B082F18
:103492000E94100F0CEA1DE00E94444BA82FB0E0DE
:1034A2001596FD01E95EF74F00810E94100F83958A
:1034B20003EA15E00E94444B082F0E94100F0CEA09
:1034C2001DE00E94444BA82FB0E01596FD01E95E75
:1034D200F74F00810E94100F839502EC15E00E94C5
:1034E200444B082F0E94100F0CEA1DE00E94444B2F
:1034F200A82FB0E01596FD01E95EF74F00810E940A
:10350200100F839501EE15E00E94444B082F0E9494
:10351200100F0CEA1DE00E94444BA82FB0E0159654
:10352200FD01E95EF74F00810E94100F83950EEEB8
:1035320012E00E94444B0E94FC0E00E016E00E9442
:10354200444B082F0E94100F0CEA1DE00E94444BCE
:10355200A82FB0E01596FD01E95EF74F00810E94A9
:10356200100F83950CE216E00E94444B082F0E9434
:10357200100F0CEA1DE00E94444BA82FB0E01596F4
:10358200FD01E95EF74F00810E94100F83950BE465
:1035920016E00E94444B082F0E94100F0CEA1DE017
:1035A2000E94444BA82FB0E01596FD01E95EF74F4B
:1035B20000810E94100F83950AE616E00E94444B98
:1035C200082F0E94100F0CEA1DE00E94444BA82F06
:1035D200B0E01596FD01E95EF74F00810E94100FE1
:1035E200839509E816E00E94444B082F0E94100FB1
:1035F2000CEA1DE00E94444BA82FB0E01596FD0195
:10360200E95EF74F00810E94100F839508EA16E0E9
:103612000E94444B082F0E94100F0CEA1DE00E94EA
:10362200444BA82FB0E01596FD01E95EF74F0081EB
:103632000E94100F839507EC16E00E94444B082F5E
:103642000E94100F0CEA1DE00E94444BA82FB0E02C
:103652001596FD01E95EF74F00810E94100F8395D8
:1036620006EE16E00E94444B082F0E94100F0CEA4F
:103672001DE00E94444BA82FB0E01596FD01E95EC3
:10368200F74F00810E94100F839505E017E00E941A
:10369200444B082F0E94100F0CEA1DE00E94444B7D
:1036A200A82FB0E01596FD01E95EF74F00810E9458
:1036B200100F839504E217E00E94444B082F0E94EA
:1036C200100F0CEA1DE00E94444BA82FB0E01596A3
:1036D200FD01E95EF74F00810E94100F839503E41C
:1036E20017E00E94444B082F0E94100F0CEA1DE0C5
:1036F2000E94444BA82FB0E01596FD01E95EF74FFA
:1037020000810E94100F839502E617E00E94444B4D
:10371200082F0E94100F0CEA1DE00E94444BA82FB4
:10372200B0E01596FD01E95EF74F00810E94100F8F
:10373200839501E817E00E94444B082F0E94100F66
:103742000CEA1DE00E94444BA82FB0E01596FD0143
:10375200E95EF74F00810E94100F839500EA17E09F
:103762000E94444B082F0E94100F0CEA1DE00E9499
:10377200444BA82FB0E01596FD01E95EF74F00819A
:103782000E94100F83950FEB17E00E94444B082F05
:103792000E94100F0CEA1DE00E94444BA82FB0E0DB
:1037A2001596FD01E95EF74F00810E94100F839587
:1037B2000EED17E00E94444B082F0E94100F0CEAF6
:1037C2001DE00E94444BA82FB0E01596FD01E95E72
:1037D200F74F00810E94100F83950DEF17E00E94B2
:1037E200444B082F0E94100F0CEA1DE00E94444B2C
:1037F200A82FB0E01596FD01E95EF74F00810E9407
:10380200100F83950CE118E00E94444B082F0E9490
:10381200100F0CEA1DE00E94444BA82FB0E0159651
:10382200FD01E95EF74F00810E94100F83950BE3C3
:1038320018E00E94444B082F0E94100F0CEA1DE072
:103842000E94444BA82FB0E01596FD01E95EF74FA8
:1038520000810E94100F83950AE518E00E94444BF4
:10386200082F0E94100F0CEA1DE00E94444BA82F63
:10387200B0E01596FD01E95EF74F00810E94100F3E
:10388200839509E718E00E94444B082F0E94100F0D
:103892000CEA1DE00E94444BA82FB0E01596FD01F2
:1038A200E95EF74F00810E94100F839508E918E046
:1038B2000E94444B082F0E94100F0CEA1DE00E9448
:1038C200444BA82FB0E01596FD01E95EF74F008149
:1038D2000E94100F839507EB18E00E94444B082FBB
:1038E2000E94100F0CEA1DE00E94444BA82FB0E08A
:1038F2001596FD01E95EF74F00810E94100F839536
:1039020006ED18E00E94444B082F0E94100F0CEAAB
:103912001DE00E94444BA82FB0E01596FD01E95E20
:10392200F74F00810E94100F839505EF18E00E9467
:10393200444B082F0E94100F0CEA1DE00E94444BDA
:10394200A82FB0E01596FD01E95EF74F00810E94B5
:10395200100F839504E119E00E94444B082F0E9446
:10396200100F0CEA1DE00E94444BA82FB0E0159600
:10397200FD01E95EF74F00810E94100F8395E4E09C
:103982000C94234E9A938A93902F80E000916609BB
:10399200109165090117D1F340E050E060E070E05A
:1039A20000916609109165090117A1F48A019B0132
:1039B200A801B9014F5F5F4F6F4F7F4F013EE3E9AF
:1039C2001E07E4E02E07E0E03E0750F3082F89913E
:1039D200999108950091660910E0F801EB56F94FAC
:1039E2000081E6E6F9E0108113951083282F30E07C
:1039F200F901E95EF74F0083992341F0082F10E0A7
:103A0200F801E95EF74F00810E94CB0D8395C4CF88
:103A12000E94124E902FA12FB22FA0939507B09320
:103A2200960700EF0093970705E5009398070FE0CC
:103A3200009399070AEA00939A0726E01DE0092FEE
:103A42000E94A549802F00916809002349F00CE8E3
:103A520010E00E94444B282F0BEC18E00E94F6491C
:103A62000AE010E00E945C0C1A2F092F0E94DE4C23
:103A72000B1711F401E001C000E0E4E00C94234EC6
:103A82000F3130F410E0F801E659F64F0081089545
:103A9200043650F00E3640F410E004561040F8019F
:103AA200E657F64F0081089500E00895A80100E06E
:103AB20001C00395083C88F410E0F901E00FF11F02
:103AC200608110E0FA01E00FF11F608310E0F9015C
:103AD200E00FF11F1081112361F70895A80100E0A2
:103AE20010E0FA01E00FF11F608110E0F901E00F30
:103AF200F11F1081611791F4039510E0FA01E00FB4
:103B0200F11F1081112339F410E0F901E00FF11FC8
:103B12001081112321F0093C18F3089500E0089563
:103B22000E940F4ED901CA01442401C04394552476
:103B3200FC01E40DF51D20812032C1F32CE3421675
:103B420008F041C05524FC01E40DF51D208122231B
:103B5200D1F120E021C05524FC01E40DF51D308196
:103B6200313670F05524FC01E40DF51D30813B37F0
:103B720038F45524FC01E40DF51D30813F75308386
:103B82005524FC01E40DF51D408130E0F801E20FFF
:103B9200F31F4083239543945524FC01E40DF51D46
:103BA2003081303350F05524FC01E40DF51D308195
:103BB2003B3718F430E1431670F240E030E0F80190
:103BC200E20FF31F4083E02FF12F0081002311F455
:103BD20000E0A6C066249EC043945524FC01E40D77
:103BE200F51D00810032C1F35524FC01E40DF51DE1
:103BF2000081002319F46394062D92C000E010E0C6
:103C020020E030E0462D50E0440F551F440F551F71
:103C1200FD01E40FF51F008311832283338342C029
:103C2200062D10E0000F111F000F111FFD01E00F04
:103C3200F11F00811181228133814AE050E060E06E
:103C420070E00E94954D462D50E0440F551F440FE1
:103C5200551FFD01E40FF51F008311832283338377
:103C62005524FC01E40DF51D008110E000531040C5
:103C7200212F220F220B322F462D50E0440F551FC9
:103C8200440F551FFD01E40FF51F408151816281F0
:103C92007381400F511F621F731F408351836283E0
:103CA200738343940CE34016A0F55524FC01E40D04
:103CB200F51D0081002321F402E0600E062D30C0C4
:103CC2005524FC01E40DF51D00810B33E1F0552470
:103CD200FC01E40DF51D00810A33A9F05524FC0115
:103CE200E40DF51D00810C3271F05524FC01E40D48
:103CF200F51D00810E3239F05524FC01E40DF51D4D
:103D02000081003281F400E25524FC01E40DF51D2E
:103D1200008363940EE1601608F45FCF6394062D6E
:103D2200E7E00C94204E00915F09002309F478CF5C
:103D32005524FC01E40DF51D0081003308F446C052
:103D42005524FC01E40DF51D00810A33F8F5062D1A
:103D520010E0000F111F000F111FFD01E00FF11FF6
:103D6200008111812281338144E00E94B14D462DB0
:103D720050E0440F551F440F551FFD01E40FF51F7E
:103D820000831183228333835524FC01E40DF51D46
:103D9200008110E000531040212F220F220B322FFE
:103DA200462D50E0440F551F440F551FFD01E40FEF
:103DB200F51F4081518162817381400F511F621F43
:103DC200731F40835183628373836BCF5524FC013D
:103DD200E40DF51D0081013408F463CF5524FC0184
:103DE200E40DF51D00810B3708F05BCF5524FC0173
:103DF200E40DF51D00810F750083062D10E0000F04
:103E0200111F000F111FFD01E00FF11F0081118131
:103E12002281338144E00E94B14D462D50E0440F8F
:103E2200551F440F551FFD01E40FF51F0083118339
:103E3200228333835524FC01E40DF51D008110E03B
:103E420007531040212F220F220B322F462D50E014
:103E5200440F551F440F551FFD01E40FF51F40810C
:103E6200518162817381400F511F621F731F408312
:103E720051836283738315CF0E94124EC801A22F11
:103E8200B1E016C008E00E94CB0D00E20E94CB0D0B
:103E920008E00E94CB0D0A2FA02FAA95002391F7CC
:103EA2002EED3DE08C0102DEA02F8C010E94EF0E70
:103EB200BB23A9F10E94FC0E102F1050C9F31A95D2
:103EC20051F3175099F0125029F0135019F01E5067
:103ED20079F319C000E0B0E0FC01EA0FFB1F008398
:103EE2009C010EED1DE0E2DD01E01AC0A13000F3FD
:103EF200AA9508E00E94CB0D00E20E94CB0D08E0DB
:103F02000E94CB0DD5CFAC3398F62A2F30E0FC01BE
:103F1200E20FF31F00830E94CB0DA395C9CF00E0EF
:103F2200E4E00C94234E0E94124E902F812F983081
:103F320050F5883040F5092F10E00F5F1F4F40E425
:103F420050E00E94544DD801082F10E00F5F1F4F20
:103F520040E450E00E94544D20E011C0422F50E056
:103F6200400F511FFA01EB52F64F3081422F50E0C1
:103F72004A0F5B1FFA01EB52F64F30832395203430
:103F820068F3092F03D0E4E00C94234E9A938A93AA
:103F9200902F973011F490E001C0939580E007C014
:103FA200182F092F50D2182F092F2BD183958F311B
:103FB200B8F31FE1092F47D21FE1092FD3D0F8012F
:103FC200EB52F64F00810E94830E10E2092F3BD282
:103FD20010E2092FC7D0F801EB52F64F00810E9480
:103FE200830E899199910895005049F00A9561F0E4
:103FF2000A9579F00A9591F00A95A9F0089504ECD2
:1040020014E10E94444B089508ED14E10E94444BD0
:10401200089506EE14E10E94444B089509EF14E15D
:104022000E94444B089509E015E10E94444B089513
:104032009A938A93802F912FE0E0F6E11491E7EFB3
:10404200F5E104910E94092F22E0082F10E00E945E
:10405200960EE1E0F6E11491E8EFF5E104910E9499
:10406200092F22E0092F10E00E94960EE2E0F6E10D
:104072001491E9EFF5E104910E94092F192F082FFD
:1040820071D00E948D0E8991999108958A93EAEFD9
:10409200F5E11491E1EFF5E104910E94092F80E02E
:1040A20004C000E20E94CB0D83958634D0F3EAEF80
:1040B200F5E11491E1EFF5E104910E94092F899154
:1040C20008959A938A939091E90980E00CC0182F81
:1040D20000911A0E0395B7D108E00E94CB0D00E2C1
:1040E2000E94CB0D83958F3190F380E00BC0182F87
:1040F200092F0395A8D108E00E94CB0D0CE70E947E
:10410200CB0D83958F3198F390931A0EEEEFF5E174
:104112001491E5EFF5E104910E94092F092F0E9405
:10412200830E899199910895093031F4133020F06A
:10413200143110F401E00895083021F41F3110F415
:1041420001E00895083030F4103211F01F3111F4FB
:1041520001E00895083020F4103210F402E00895CE
:1041620000E00895682F202F812F222371F48F31D0
:1041720038F4082F10E0000F111F00501E4F39C0F5
:10418200082F10E0015E1D4F34C08F3149F4022F19
:1041920010E040E450E00E94544D025C1F4F29C0E1
:1041A200803249F4022F10E040E450E00E94544D66
:1041B200015C1F4F1EC0283029F4082F10E0005E5A
:1041C2001F4F17C0293029F4082F10E0055F1F4F39
:1041D20010C0022F10E00150104040E450E00E9455
:1041E200544D980102E0809F8001020F131F005C72
:1041F2001F4F003422E0120710F000E010E0862F7B
:1042020008959A938A93902F812F8F3108F042C09C
:10421200182F092FA7DFF801EB52F64F20813181C9
:10422200203004E0300748F0182F092F9BDFF801F7
:10423200EB52F64F018107FF0BC0182F092F92DFB7
:10424200F801EB52F64F008111810E948D0E22C0BF
:10425200182F092F87DFF801EB52F64F018105FF76
:104262000DC00FE30E94CB0D0FE30E94CB0D0FE3B5
:104272000E94CB0D0FE30E94CB0D0CC00DE20E94F9
:10428200CB0D0DE20E94CB0D0DE20E94CB0D0DE293
:104292000E94CB0D8991999108959A938A930091E6
:1042A200DA0C002351F000E09FDE0E94FC0E09357B
:1042B20021F0093711F000E085C0E8EDFCE0008153
:1042C200118120E030E040E052E060E070E00E94C6
:1042D200954DA801B901405050426F4F7F4F90E079
:1042E20000E010E018C0080122243324040E151E39
:1042F200261E371EF001322D3BBF069020E02BBF59
:10430200F801EB52F64F0082F801EB52F64F208192
:10431200920F0F5F1F4F003022E0120720F380E060
:104322000DC020E030E402E0809F800100501E4F6B
:10433200F801EB52F64F2083318383958F3180F55C
:10434200082F10E0F801E659F64F0081002349F3E7
:1043520018E1082F0E94DE4C013081F41EE1082F83
:104362000E94DD2E22E0829F20E0020E22E0121E39
:10437200F001EB52F64F00831183DFCF14E2082FD6
:104382000E94DD2E0060106222E0829F20E0020E79
:1043920022E0121EF001EB52F64F00831183CDCFC3
:1043A2009F3F21F40091E909083008F00ED000E0A7
:1043B2000093DA0C0091EC09053018F000E000934C
:1043C200EC0901E08991999108953B2F2A2FE0E0B1
:1043D200F0E006C000E0DF01AB52B64F0C9331961D
:1043E200E03200E0F007B0F3E0E2F0E006C005E5FD
:1043F200DF01AB52B64F0C933196E03400E0F00788
:10440200B0F3E0E4F0E009C000E010E4DF01AB52F9
:10441200B64F0D931C9311973296E03002E0F007ED
:1044220098F300E00093E90901E00093E40900E257
:104432000093EB0900E20093ED0900E00093E2092A
:10444200A22FB32F08959A938A936297602F212FF8
:10445200CE010896ECECFCE930E08C014AE050E039
:104462000E94F54DCE01E6EDFCE930E08C0148E01A
:1044720050E00E94F54D203211F02F3151F4239576
:10448200122FFE0170E0E60FF71F00810E94092F34
:1044920010C02F3158F42395122FFE01389670E088
:1044A200E60FF71F00810E94092F03C001E20E945C
:1044B200CB0D62968991999108958A93802F03C0BA
:1044C20000E20E94CB0D082F802F8A950023C1F7AE
:1044D200899108950E94134E80E005C00CE810E017
:1044E2000E94444B83958C33C8F311E001E00E9493
:1044F200092F05E21FE00E94444B0FE31FE00E94D8
:10450200444B07E2DADF0AE51FE00E94444B07E66C
:104512001FE00E94444B07E2D0DF02E81FE00E9446
:10452200444B09E81FE00E94444B07E2C6DF04EA5D
:104532001FE00E94444B02EB1FE00E94444B07E243
:10454200BCDF0DEC1FE00E94444B0BED1FE00E940C
:10455200444B07E2B2DF06EF1FE00E94444B04E047
:1045620010E10E94444B07E2A8DF0FE110E10E9434
:10457200444B0DE210E10E94444B07E29EDF08E447
:1045820010E10E94444B06E510E10E94444B07E211
:1045920094DF01E710E10E94444B0FE710E10E9413
:1045A200444B07E28ADF0AE910E10E94444B08EA21
:1045B20010E10E94444B07E280DF03EC10E10E940D
:1045C200444B01ED10E10E94444B07E276DF0CEE12
:1045D20010E10E94444B0AEF10E10E94444B07E2B3
:1045E2006CDF05E111E10E94444B03E211E10E94FC
:1045F200444B07E262DF0EE311E10E94444B0CE4FC
:1046020011E10E94444B07E258DF07E611E10E94E4
:10461200444B05E711E10E94444B07E24EDF00E9FB
:1046220011E10E94444B0EE911E10E94444B07E262
:1046320044DF09EB11E10E94444B07EC11E10E94B7
:10464200444B07E23ADF02EE11E10E94444B00EFD5
:1046520011E10E94444B07E230DF0BE012E10E94BD
:10466200444B09E112E10E94444B07E226DF04E3D6
:1046720012E10E94444B02E412E10E94444B0DE518
:1046820012E10E94444B08E712E10E94444B03E905
:1046920012E10E94444B0EEA12E10E94444B09ECE3
:1046A20012E10E94444B04EE12E10E94444B0FEFD0
:1046B20012E10E94444B0AE113E10E94444B05E3DC
:1046C20013E10E94444B00E513E10E94444B0BE6C8
:1046D20013E10E94444B06E813E10E94444BE8EDCB
:1046E200FCE000811181012B29F406E214E10E9411
:1046F200444B04C007ED13E10E94444B05E714E16B
:104702000E94444B80E001C083958132F8F490E02E
:1047120006C0A23019F4182F092F73DD9395933137
:1047220098F7182F092F00DDA02FAA23B9F3182F0D
:10473200092F89DEA13069F7182F092F13DDF8013F
:10474200EB52F64F00810E94830EE8CFBADCEBEF0A
:10475200F5E11491E2EFF5E104910E94092F05EDD4
:1047620019E00E94EF0EECEFF5E11491E3EFF5E1B1
:1047720004910E94092FE8EDFCE0008111810E9462
:104782008D0EEDEFF5E11491E4EFF5E104910E9455
:10479200092FE8EDFCE00081118120E030E040E0EB
:1047A20052E060E070E00E94954D005010422F4FA1
:1047B2003F4F0E94DE0EE3E00C94244E0E94094E0D
:1047C200EF97EA97DA95BE0164527F4FEEEDFCE96E
:1047D20030E08B0141E250E00E94F54DA0E0BA2F9B
:1047E200BA2ECA2E24EF3FE0A9010E94364D0535AC
:1047F20011F40C94262E1A2F0B2F1ADC1A2F0B2FC2
:1048020022DE9090E90900915F09002319F000E18E
:10481200A02E02C00AE0A02E0E94FC0E902F9B3117
:10482200D9F50E94FC0E902F9B3519F40E94FC0EC4
:10483200902F943421F4BB2389F0BA950FC093349E
:1048420011F4B3950BC0913421F4AA2339F0AA953F
:1048520005C0923419F4A03208F4A395FE01E45283
:10486200FF4F0A2F10E0E00FF11F00810B1738F401
:10487200FE01E452FF4FB0E0EA0FFB1FB081BC150E
:1048820021F4AB1511F40C94C02E1A2F0B2FD0DB90
:10489200CB2EBA2E0C94C02E903209F044C01A2F9F
:1048A2000B2F42DC023011F00C94C02E80E090E21B
:1048B2001A2F0B2F57DCF801EB52F64F00811181B2
:1048C2000827192700831183BB2329F58A2F02E0C9
:1048D200809F800100501E4FF801EB52F64F01817C
:1048E20005FD16C090E0FC01E659F64F0081002359
:1048F20079F014E2082F0E94DD2E22E0829F20E050
:10490200020E22E0121EF001EB52F64F00831183D9
:104912000A2F0E947E391A2F0B2F73DC01E00093BD
:10492200DA0C0C94C02E9D3509F04CC01A2F0B2FB7
:104932008ADD1A2F0B2FF8DB0130B9F41A2F0B2F57
:1049420011DCF801EB52F64F0081039500831A2F18
:104952000B2F08DCF801EB52F64F00810E94830E08
:1049620001E00093DA0C0C94C02E023011F00C948A
:10497200C02E1A2F0B2FF6DBF801EB52F64F0081F7
:1049820011810F7F13700F3F23E0120711F40C9473
:10499200C02E1A2F0B2FE6DBF801EB52F64F0081E7
:1049A20011810F5F1F4F008311831A2F0B2F29DCF8
:1049B200BB2319F40A2F0E947E3901E00093DA0C1E
:1049C2000C94C02E9B3509F04AC01A2F0B2F3BDDE9
:1049D2001A2F0B2FA9DB0130B9F41A2F0B2FC2DBD0
:1049E200F801EB52F64F00810A9500831A2F0B2F24
:1049F200B9DBF801EB52F64F00810E94830E01E011
:104A02000093DA0C0C94C02E023011F00C94C02EDC
:104A12001A2F0B2FA7DBF801EB52F64F0081118101
:104A22000F7F1370012B11F40C94C02E1A2F0B2F31
:104A320099DBF801EB52F64F0081118101501040D1
:104A4200008311831A2F0B2FDCDBBB2319F40A2FEF
:104A52000E947E3901E00093DA0C0C94C02E9D373F
:104A620009F050C01A2F0B2F5FDB0130B9F41A2F57
:104A72000B2F78DBF801EB52F64F00810A0D008311
:104A82001A2F0B2F6FDBF801EB52F64F00810E94B9
:104A9200830E01E00093DA0C0C94C02E023011F068
:104AA2000C94C02E1A2F0B2F5DDBF801EB52F64F40
:104AB200008111810F7F13702FEF33E04A2D50E0F8
:104AC200241B350B0217130710F00C94C02E8A2DED
:104AD20090E01A2F0B2F46DBF801EB52F64F0081C4
:104AE2001181080F191F008311831A2F0B2F89DBE5
:104AF200BB2319F40A2F0E947E3901E00093DA0CDD
:104B02000C94C02E9B3709F04CC01A2F0B2F0CDBD4
:104B12000130B9F41A2F0B2F25DBF801EB52F64FB7
:104B220000810A1900831A2F0B2F1CDBF801EB52AC
:104B3200F64F00810E94830E01E00093DA0C0C9480
:104B4200C02E023011F00C94C02E1A2F0B2F0ADB4C
:104B5200F801EB52F64F008111810F7F13702A2D5D
:104B620030E00217130710F40C94C02E8A2D90E047
:104B72001A2F0B2FF7DAF801EB52F64F0081118151
:104B8200081B190B008311831A2F0B2F3ADBBB234F
:104B920019F40A2F0E947E3901E00093DA0C0C947A
:104BA200C02E74DA903360F09B3750F4092F0E94C4
:104BB200CB0D98A721E08E01085D1F4F5DD905C07E
:104BC20020E08E01085D1F4F57D900E00883AE0137
:104BD200485D5F4F9E012C593F4F8E010E94911DEF
:104BE200902F992311F40C94C02E28E935E08E0100
:104BF2000E946F1D002351F001E000935F09A0E0C5
:104C0200BA2F1A2F0B2F14DA0C94C02E24E935E098
:104C12008E010E946F1D002351F000E000935F0996
:104C2200A0E0BA2F1A2F0B2F03DA0C94C02E2BE41C
:104C320036E08E010E946F1D002341F04BDCA0E0A4
:104C4200BA2F1A2F0B2FF4D90C94C02E27E436E07A
:104C52008E010E946F1D002339F427EE35E08E018C
:104C62000E946F1D002391F0EAEFF5E11491E1EF4C
:104C7200F5E104910E94092F0E94200F2BDCA0E095
:104C8200BA2F1A2F0B2FD4D90C94C02E22E436E05F
:104C92008E010E946F1D0023B1F0933021F002E0DB
:104CA200A3D90C94C02EFE01FF9605A116A127A13F
:104CB20030A5B02FFE01FF9601A512A523A534A5AC
:104CC200A02F0C94C02E2DE336E08E010E946F1DA2
:104CD200002339F42BE336E08E010E946F1D00237E
:104CE20049F1E8EDFCE0208131812F3700E0300707
:104CF200E8F4E8EDFCE0008111810F5F1F4F0083B3
:104D02001183CBDA002341F0E5DBA0E0BA2F1A2FA2
:104D12000B2F8ED90C94C02EE8EDFCE0008111819E
:104D220001501040008311830C94C02E01E05CD925
:104D32000C94C02E24E336E08E010E946F1D0023E6
:104D420039F422E336E08E010E946F1D002321F127
:104D5200E8EDFCE000811181012BD9F0E8EDFCE0E7
:104D620000811181015010400083118396DA0023E3
:104D720039F0B0DBA0E0BA2F1A2F0B2F59D9FFC799
:104D8200E8EDFCE0008111810F5F1F4F008311836A
:104D9200F6C701E029D9F3C72DE236E08E010E9461
:104DA2006F1D002339F42BE236E08E010E946F1D45
:104DB200002399F1923019F002E016D9E0C7FE0102
:104DC200FF9605A116A127A130A5003840E01407DF
:104DD20040E0240740E03407E8F4E8EDFCE080819D
:104DE2009181FE01FF9605A116A127A130A5E8ED4C
:104DF200FCE00083118351DA002339F06BDBA0E081
:104E0200BA2F1A2F0B2F14D9BAC7E8EDFCE0808312
:104E12009183B5C701E0E8D8B2C726E236E08E0139
:104E22000E946F1D0023D1F1923019F002E0DCD80C
:104E3200A6C7FE01FF9605A116A127A130A500383D
:104E420040E0140740E0240740E0340720F5E8ED95
:104E5200FCE080819181FE01FF9605A116A127A1A8
:104E620030A5E8EDFCE00083118317DA002371F02E
:104E7200E8EDFCE0808391832DDBA0E0BA2F1A2FAE
:104E82000B2FD6D801E00093DA0C79C7E8EDFCE0ED
:104E92008083918374C701E0A7D871C72AE536E001
:104EA2008E010E946F1D0023E1F00091DA0C0023B5
:104EB20089F000E099D80E94FC0E902F993519F0E4
:104EC200993709F05CC704E110E00E945C0C08E02D
:104ED20001BD55C704E110E00E945C0C08E001BD71
:104EE2004EC721E236E08E010E946F1D002319F1A8
:104EF2000AE30E94CB0D20E08E01085D1F4F0E9445
:104F02003D1F002361F000E00DAB9E01285D3F4F85
:104F120005ED19E00E94571D01E00093DA0CEBEF5A
:104F2200F5E11491E2EFF5E1049172D705ED19E094
:104F32000E94EF0E24C72EE136E08E010E946F1D03
:104F4200002309F482C09130A9F580E08F3108F086
:104F520016C702E0809F00E0000E02E0101EF00182
:104F6200EB52F64F018105FF23C090E0FC01E659A8
:104F7200F64F00810023E1F021E018E1082F0E94A2
:104F8200034D14E2082F18D722E0829F20E0020E80
:104F920022E0121EF001EB52F64F00831183082F1C
:104FA2000E947E39182F00E04EDA182F00E029D92E
:104FB2008395CCCF44245524E92FF0E031974E1647
:104FC2005F060CF0DCC6FE01EC59FF4F042D10E029
:104FD200000F111F000F111FE00FF11F008111813F
:104FE20022813381802F02E0809F00E0000E02E0E8
:104FF200101EF001EB52F64F018105FF24C0082F6D
:1050020010E0F801E659F64F00810023E1F021E0BB
:1050120018E1082F0E94034D14E2082FCDD622E09A
:10502200829F20E0020E22E0121EF001EB52F64FA8
:1050320000831183082F0E947E39182F00E003DAC3
:10504200182F00E0DED84394B6CF2AE136E08E0175
:105052000E946F1D002309F460C0913021F580E0A9
:105062008F3108F08CC690E0FC01E659F64F0081C2
:105072000023B9F020E018E1082F0E94034D02E05E
:10508200809F00E0000E02E0101EF001EB52F64F8E
:10509200018100620183182F00E0D5D9182F00E0AA
:1050A200B0D88395DDCF44245524E92FF0E0319721
:1050B2004E165F060CF063C6FE01EC59FF4F042D3D
:1050C20010E0000F111F000F111FE00FF11F0081F0
:1050D200118122813381802F082F10E0F801E659D7
:1050E200F64F00810023B9F020E018E1082F0E945A
:1050F200034D02E0809F00E0000E02E0101EF0016E
:10510200EB52F64F018100620183182F00E09BD918
:10511200182F00E076D84394C7CF22E136E08E0103
:105122000E946F1D002309F466C0913009F048C047
:105132000091FE0C1091FD0C011709F020C608EC3D
:1051420010E00E945C0C0E944720EAEFF5E1149106
:10515200E1EFF5E104915CD612E206E60E94DE4C34
:105162000E94830E00E20E94CB0D13E206E60E942B
:10517200DE4C0E94830E00E20E94CB0D14E206E692
:105182000E94DE4C0E94830E0CE20E94CB0D12E2C2
:1051920005E60E94DE4C0E94830E00E20E94CB0DC7
:1051A20013E205E60E94DE4C0E94830E00E20E949A
:1051B200CB0D14E205E60E94DE4C0E94830EB8CFAE
:1051C200923009F0DCC580E007C000E090E0FC010D
:1051D200E455F24F008383958F31B8F3FE01FF96B9
:1051E20005A116A127A130A50093D70C07E115E16F
:1051F2000E94444BC4C52DE036E08E010E946F1D13
:10520200002339F423E936E08E010E946F1D00234A
:10521200C1F0FE01FF9605A116A127A130A592308B
:1052220021F002E00E94F51FAAC5083020F004E038
:105232000E94F51FA4C50093E90901E00093DA0C6E
:105242009EC52EE836E08E010E946F1D002399F163
:10525200933021F002E00E94F51F91C5FE01FF96F6
:1052620005A116A127A130A5802FFE01FF9601A559
:1052720012A523A534A5902F983010F4883020F081
:1052820004E00E94F51F7BC50AE30E94CB0D082FA4
:105292000E94830E0DE20E94CB0D0EE30E94CB0D05
:1052A200092F0E94830E182F092F0E94941F01E0DC
:1052B2000093DA0C64C52DE735E08E010E946F1D64
:1052C200002341F428E735E08E010E946F1D002380
:1052D20009F488C0933020F002E00E94F51F4FC508
:1052E200913019F40091E90906C0FE01FF9605A16B
:1052F20016A127A130A5073020F004E00E94F51F77
:105302003EC5E8EDFCE020813181232B41F4109170
:10531200E909133020F004E00E94F51F30C59230F5
:1053220039F417E00E94941F01E00093DA0C19C0CF
:105332009130A1F40091E909073080F417E000915F
:10534200E9090E94941FE5EDF9E004890395048BB5
:105352000E94622001E00093DA0C03C004E00E9484
:10536200F51FE8EDFCE000811181012B09F007C572
:105372000091E909013029F00091E909023009F0B0
:10538200FEC400E410E020E830E040EC50E080E0B1
:105392001EC062E0869F020E131EF001EB52F64F12
:1053A2002080318062E0869F000E111EF001EB52D8
:1053B200F64F60817181261A370A62E0869F040ED9
:1053C200151EF001EB52F64F2082318283958F3108
:1053D20000F30E94472003E00E94F51F02E00E94B2
:1053E200C71FCDC427E836E08E010E946F1D00233F
:1053F20039F42BE036E08E010E946F1D0023E9F1A3
:10540200923029F5FE01FF9605A116A127A130A52C
:10541200802F873020F004E00E94F51FB0C4009175
:10542200E909801770F4E5EDF9E004890A95048B27
:105432000E94622006C0182F1395082F0E94941F05
:1054420083958630C0F301E00093DA0C98C4913062
:1054520009F095C40091E909013058F0E5EDF9E051
:1054620004890A95048B0E94622001E00093DA0C01
:1054720086C404E00E94F51F82C420E836E08E0153
:105482000E946F1D002339F42EE736E08E010E9440
:105492006F1D002389F1FE01FF9605A116A127A128
:1054A20030A5802F923021F002E00E94F51F67C4E0
:1054B200873020F004E00E94F51F61C406E0402E10
:1054C20006C0142D1A95042D0E94941F4A94841527
:1054D200C0F317E0082F0E94941F0091E90980177A
:1054E20038F4E5EDF9E004890395048B0E9462200B
:1054F20001E00093DA0C43C42DEB35E08E010E94EB
:105502006F1D002379F0923048F0FE01FF9605A14D
:1055120016A127A130A50E94974031C401E00E9444
:1055220097402DC42FE435E08E010E946F1D0023A9
:1055320041F42DE435E08E010E946F1D002309F431
:1055420061C0FE01FF9605A116A127A130A5402E3C
:10555200923021F002E00E94F51F11C407E04016CC
:1055620020F004E00E94F51F0AC499E580E01DC006
:10557200082F10E0F801E659F64F00810023A1F050
:10558200042D10E040E450E00E94544D22E0829F3E
:10559200000E111E00E4000E00E0101EF001EB529E
:1055A200F64F018106FD9EE483958F3108F3009149
:1055B200E909401640F0993531F400E00E94F51FE8
:1055C2000E94FC0E902F993519F0993709F0D7C334
:1055D200EFEFF5E11491E6EFF5E1049119D4042D12
:1055E2000E94830E07E00E94C71F142D07E00E944D
:1055F200941F80E08F3108F0C2C3082F0E947E39C9
:105602008395F8CF29E736E08E010E946F1D0023B3
:1056120009F4BAC0E8EDFCE040805180913061F4B9
:10562200E8EDFCE00081118120E030E0FE01FF9610
:1056320005A316A327A330A7E4EDFDE02081318165
:10564200273302E0300738F023E333E012E20EEFB3
:105652000E940B4D06C02FEF33E012E20EEF0E94C4
:105662000B4D00E010E0E8EDFCE00083118380E0E8
:105672000CC022E0829F20E0020E22E0121EF00106
:10568200EB52F64F0083118383958F3100F590E042
:10569200FC01E659F64F00810023B1F318E1082F0F
:1056A2000E94DE4C013021F41EE1082F85D303C095
:1056B20014E2082F81D3003020E41207D1F60DED59
:1056C2001DE00E94444B082F0E94830EDDCFE8EDBF
:1056D200FCE040825182FE01FF9605A116A127A19E
:1056E20030A5A6D407C001E00093DB0C05EF1DE056
:1056F2000E94444B0091DD0C0023A1F00091FE0CAE
:105702001091FD0C0117B1F30E94FC0E0B3159F3FD
:105712000D3081F702E00093DB0C0CEF1DE00E94DC
:10572200444BE8CF07E115E10E94444B04EF11E03E
:105732000E945C0C80E00CC022E0829F20E0020EFE
:1057420022E0121EF001EB52F64F00831183839583
:105752008F31B0F490E0FC01E659F64F008100234E
:10576200B1F31EE1082F28D3003020E4120721F7FD
:105772000DED1DE00E94444B082F0E94830EE7CFDF
:1057820007E00E94C71FFBC225E736E08E010E9498
:105792006F1D002309F457C0923051F4FE01FF96A9
:1057A20005A116A127A130A5003024E0120720F0A0
:1057B20002E00E94F51FE3C21A2F0B2F0E9424223F
:1057C2001A2F0B2F0E9495200130E9F4FE01FF965B
:1057D20005A116A127A130A5802F1A2F0B2F0E94F9
:1057E200B320F801EB52F64F80831A2F0B2F0E9441
:1057F200B320F801EB52F64F00810E94830E01E0C4
:105802000093DA0CBCC2023009F0B9C2FE01FF9665
:1058120005A116A127A130A5C8011A2F0B2F0E949E
:10582200B320F801EB52F64F808391831A2F0B2F8E
:105832000E940221BB2319F40A2F0E947E3901E043
:105842000093DA0C9CC22EE636E08E010E946F1D98
:10585200002341F42CE636E08E010E946F1D0023E6
:1058620009F443C1BE01605F7F4FEFEFFCE930E016
:105872008B0148E150E00E94F54D923071F4FE0137
:10588200FF9605A116A127A130A5073040E0140715
:1058920040E0240740E0340720F002E00E94F51FB8
:1058A2006EC201E00093DA0CFE01FF9605A116A17B
:1058B20027A130A5102F07E00E94941F40E452EE6A
:1058C20060E070E080E03AC002E0809F8001212F1A
:1058D200220F220B322F040F151F261F371F0F5FB7
:1058E2001F4F2F4F3F4FF801322F3BBF069000E072
:1058F2000BBF302C222402E0809F8001212F220F37
:10590200220B322F040F151F261F371FF801322FCB
:105912003BBF0690202D00E00BBF30E0220D331D6F
:105922002F7F3370FE01E55CFE4F082F10E0000F61
:10593200111FE00FF11F2083318383958F3120F2F5
:10594200FE01FF9605A116A127A130A540E450E073
:105952000E94544D005C1F4F80E026C022E0829FCF
:10596200000E111E21E0020E20E0121EF001EB5289
:10597200F64F508140E022E0829F000E111EF0019E
:10598200EB52F64F208130E0240F351F2F7F33700A
:10599200FE01E350FF4F482F50E0440F551FE40F24
:1059A200F51F2083318383958F31C0F280E068C078
:1059B200FE01E55CFE4F082F10E0000F111FE00F03
:1059C200F11F208131812F7F33708E0103501F4FD1
:1059D200FE01709690E0E80FF91F408150E0440FFD
:1059E200551F040F151FE02FF12F008111810F7F2A
:1059F2001370201B310B8E01055C1E4FFE01709649
:105A020090E0E80FF91F408150E0440F551F040F4A
:105A1200151FE02FF12F008111810F7F1370020FEC
:105A2200131F22E0829F20E0020E22E0121EF001EC
:105A3200EB52F64F008311838E0103501F4FFE017C
:105A4200709690E0E80FF91F208130E0220F331F9B
:105A5200020F131FE02FF12F0081118100701C7FB4
:105A620022E0829F20E0020E22E0121EF001EB52A1
:105A7200F64F20813181202B312B20833183839576
:105A82008F3138F590E0FC01E659F64F0081002392
:105A9200B1F3FE01709690E0E80FF91F00810F3F0D
:105AA20009F086CFFE01E350FF4F082F10E0000FF0
:105AB200111FE00FF11F0081118122E0829F20E07F
:105AC200020E22E0121EF001EB52F64F0083118308
:105AD200D6CF07E00E94C71F80E08F3108F04FC188
:105AE200082F0E947E398395F8CF28E636E08E0192
:105AF2000E946F1D0023C1F000E00E94F51F0E946A
:105B0200FC0E093519F0093709F039C10E94E62166
:105B12000E946B22A0E0BA2F1A2F0B2F0E9419208D
:105B220001E00093DA0C2BC123E636E08E010E94DD
:105B32006F1D002341F42FE536E08E010E946F1D98
:105B4200002309F418C110E088242FEF3FE0A901D7
:105B52000E94364D22EF3FE0A9010E94424D01E131
:105B62002FEF3FE0A9010E94424D80E090E006C085
:105B7200FC01EB52F64F0081100F0196803002E0DB
:105B82009007B0F30091F409011B0A950093F40900
:105B92000EE20E94CB0D80E090E00BC0FC01EB52C4
:105BA200F64F00819C012050384FA9010E94424DBE
:105BB2000196803002E0900788F30091130C20E0F8
:105BC2003AE0A9010E94424D0091140C21E03AE012
:105BD200A9010E94424D80E090E001C00196803010
:105BE20002E0900770F49C012050384FA9010E94F6
:105BF200364DFC01EB52F64F1081011779F38824E0
:105C02008394E8EDFCE00081118125EF3FE0A901DA
:105C12000E94424D882009F075C025EF3FE0A9019E
:105C22000E94364DE8EDFCE020813181021709F037
:105C320069C00AEA24EF3FE0A9010E94424D08E050
:105C420001BD04EF11E00E945C0C25EF3FE0A901C9
:105C52000E94364D10E0E8EDFCE000831183E8ED90
:105C6200FCE0008111810F7F107000831183882472
:105C72000FEF24EF3FE0A9010E94424DE8EDFCE066
:105C82000081118120E030E040E052E060E070E00D
:105C92000E94954D2801390100E0400E00EE501E91
:105CA20000E0601E00E0701E80E090E001C00196FE
:105CB200803002E09007C0F49C012050384FA901C7
:105CC2000E94364D602F8C0120E030E0040D151D3E
:105CD200261D371DF801322F3BBF069000E00BBF97
:105CE200601529F302E0802E20E03AE0A9010E942B
:105CF200364D0093130C21E03AE0A9010E94364D83
:105D02000093140C8820F9F40E944E210091EA09B4
:105D1200002361F0E8EDFCE0008111812091EA09A5
:105D220030E020503F4FA9010E94424D07E115E1AA
:105D32000E94444B0E946B22A0E0BA2F1A2F0B2F15
:105D42000E94192009C005ED1DE00E94444B00E3AA
:105D5200800E082D0E94CB0D00E00093DA0C22EF9A
:105D62003FE0A9010E94364D2FEF3FE0A9010E94BA
:105D7200424DAD9804C008EE1DE00E94444B0091D4
:105D8200E909091599F00091E909013F20F000E0C5
:105D92000093E90907C00091E909083018F007E00B
:105DA2000093E9090E9462209090E9091A2F0B2FB3
:105DB2000E9424220C940D249A938A93802F082FF8
:105DC2000E94ED4C0F3F2FEF120719F400E012E092
:105DD2001CC0E8EDFCE020813181232B51F090E0E2
:105DE200880F991FFC01EB56F64F20813181021B6F
:105DF200130B212F27FF03C000E010E006C0003084
:105E020024E0120710F00FEF13E0899199910895A1
:105E12009A938A93902F812F02E00E94CB0D0BE17F
:105E22000E94CB0D0BE50E94CB0D8A3038F0082F73
:105E32004AE00E94464D005D0E94CB0D082F4AE0C9
:105E42000E94464D042F005D0E94CB0D0BE30E9481
:105E5200CB0D9A3038F0092F4AE00E94464D005D82
:105E62000E94CB0D092F4AE00E94464D042F005D8F
:105E72000E94CB0D06E60E94CB0D8991999108955F
:105E82009A938A93FA93EA933A922A921A920A92EC
:105E92007A936A935A934A933A932A931A930A9358
:105EA2008FB79BB700E00BBF78940091DD0C002305
:105EB20049F00091DC0C002321F004E20E94CB0D9A
:105EC20001C0CED0EFEEFCE0008111810F5F1F4FC9
:105ED2000083118300911B0E102F139510931B0E3C
:105EE2000F70002309F06EC0E1EFFCE00081118128
:105EF200012B41F0E1EFFCE00081118101501040E3
:105F0200008311830091EE0C002349F0EEEEFCE0D9
:105F120000810A95008308E015B3102715BBAA9AE1
:105F2200A99A24B135B10091DC0D10E00370107014
:105F3200000F111FF801EC52F24F20833183ECED78
:105F4200FDE0008103950083037007B900911C0EE8
:105F5200102F139510931C0E0770002399F5EBEC8C
:105F6200FDE00081039500830E94F342879B2AC0D3
:105F7200969B28C00091E80C002321F500919A001D
:105F82000F7700939A00959A96980FE113E00150CB
:105F92001040E9F700C0000000919B00102F17FF8E
:105FA2000AC000919C00053531F404E110E00E9422
:105FB2005C0C08E001BD969A959800919A000068E1
:105FC20000939A00EDEDFDE0008107FF0CC0009107
:105FD2001B0E002311F4A89815C000911B0E083067
:105FE20089F4A89A0FC000911B0E1091DD0D1023A9
:105FF200112341F40091DD0D002321F001E015B3DE
:10600200102715BB00E00093100D9BBF8FBF0991B5
:1060120019912991399149915991699179910990EF
:10602200199029903990E991F9918991999118954E
:106032009A938A93C80120E030E010E20EEF0E94AA
:106042000B4DEAEEFCE08083918301E00093E90CC2
:106052000093DD0C00E00093DB0C89919991089587
:106062000E94084E24970091E90C002309F44DC0C8
:1060720000E000935E1000E010E0E4E5F0E1008350
:106082001183E2E5F0E100831183E6E5F0E10083AC
:10609200118300E00093A50C03E000935C10CC2474
:1060A20031C002E0C09E800100501E4FF801EB5249
:1060B200F64F208131810C2D10E0000F111FF801E5
:1060C200E75DF04F2083318300E010E02C2D30E0BB
:1060D200220F331FF901E151F04F008311832C2D60
:1060E20030E0220F331FF901EF5DF14F008311837E
:1060F2002C2D30E0220F331FF901E355F04F0083BE
:106102001183C3940FE1C01660F2E2E5F0E1008171
:106112001181E4E5F0E1208131810217130708F0D3
:106122000CC3E2E5F0E1008111810F5F1F4F008394
:106132001183E7EDFCE0008100FF86C0EFEEFCE09A
:10614200008111810370002309F059C002E200931B
:10615200950703E00093960722E012E006E60E940C
:10616200204A002331F000911C0810911D089091E3
:106172001E0800915F10000F00935F10EFE5F0E141
:10618200008101FF08C09B3068F0EFE5F0E100817B
:106192000160008307C0933328F0EFE5F0E100814E
:1061A2000160008302E20093950703E000939607E3
:1061B20022E012E005E60E94204A002331F000911D
:1061C2001C0810911D0880911E0800916010000F9C
:1061D20000936010E0E6F0E1008101FF08C08B301F
:1061E20098F1E0E6F0E10081016000832DC0833385
:1061F20058F1E0E6F0E100810160008325C0EFEE96
:10620200FCE0008111810370013061F408E2009327
:10621200950704E00093960722E012E007E60E9449
:10622200204A12C0EFEEFCE00081118103700230BF
:1062320059F404E30093950704E00093960722E0E3
:1062420012E007E60E94204A00915C10033009F434
:1062520074C280E00CE190E0FC01EB56F84F008341
:10626200839504E090E0FC01EB56F84F00838395A0
:10627200CC244CC001E010E02C2D30E0205E3F4FDA
:10628200F901EA56F34F408142954F700E94644DE6
:1062920090E0FC01EB56F84F0083839501E010E09B
:1062A2002C2D30E0205E3F4FF901EA56F34F40813A
:1062B2004F700E94644D90E0FC01EB56F84F008352
:1062C200839502E0C09E00E0000E02E0101EF00185
:1062D200EB52F64F0081118190E0FC01EB56F84F32
:1062E2000083839502E0C09E00E0000E02E0101ED3
:1062F200F001EB52F64F00811181012F10E090E086
:10630200FC01EB56F84F00838395C3940FE1C0164E
:1063120008F00EC2DD24F601E659F64F0081002393
:10632200A1F300915C10002309F092C00C2D10E043
:10633200000F111FF801E559F04F008111812C2D3A
:1063420030E0220F331FF901E355F04F20813181F4
:10635200021B130B212F220F220B322FE2E5F0E159
:106362004081518160E070E00E94954DE4E5F0E1EA
:106372004081518160E070E00E94DF4D2C2D30E0C1
:10638200220F331FF901E355F04F40815181400F35
:10639200511F2C2D30E0220F331FF901E151F04F34
:1063A200408351832C2D30E0220F331FF901E35536
:1063B200F04F2081318115950795020F131F212F70
:1063C200220F220B322FE2E5F0E14081518160E0A1
:1063D20070E00E94954D40E950E060E070E00E945C
:1063E200954D4FE050E060E070E00E94DF4D012FDC
:1063F200122F232F330F330B2595179507952C2D2D
:1064020030E0220F331FF901EB55F14F0083118366
:106412000C2D10E0000F111FF801E951F14F2081FE
:1064220031810C2D10E0000F111FF801EB55F14FD7
:1064320000811181020F131F22E0C29E20E0020E92
:1064420022E0121EF001EB52F64F0083118310C1BD
:1064520000915C10013009F046C00C2D10E0000FD5
:10646200111FF801E951F14FA081B1810C2D10E00B
:10647200000F111FF801ED59F14F00811181212FF9
:10648200220F220B322FE2E5F0E14081518160E0E0
:1064920070E00E94954DE4E5F0E14081518160E0B9
:1064A20070E00E94DF4D0A0F1B1F22E0C29E20E017
:1064B200020E22E0121EF001EB52F64F008311830E
:1064C2000C2D10E0000F111FF801E559F04F20814B
:1064D20031810C2D10E0000F111FF801E151F04F36
:1064E20020833183C5C0DD24F601EF5CFF4E0081BD
:1064F200002309F078C00C2D10E0000F111FF801E5
:10650200E355F04F00811181119501951040212F23
:10651200220F220B322FE2E5F0E14081518160E04F
:1065220070E00E94954DE4E5F0E14081518160E028
:1065320070E00E94DF4D2C2D30E0220F331FF90155
:10654200E355F04F40815181400F511F2C2D30E017
:10655200220F331FF901E151F04F408351832C2D5B
:1065620030E0220F331FF901E951F14FA081B181CF
:106572002C2D30E0220F331FF901E355F04F20811B
:10658200318115950795020F131F212F220F220B20
:10659200322FE2E5F0E14081518160E070E00E943B
:1065A200954D40E950E060E070E00E94954D4FE06B
:1065B20050E060E070E00E94DF4D012F122F232F88
:1065C200330F330B2595179507950A0F1B1F22E0F2
:1065D200C29E20E0020E22E0121EF001EB52F64FA4
:1065E2000083118345C00C2D10E0000F111FF8012C
:1065F200E951F14FA081B1810C2D10E0000F111F64
:10660200F801ED59F14F00811181212F220F220B48
:10661200322FE2E5F0E14081518160E070E00E94BA
:10662200954DE4E5F0E14081518160E070E00E9427
:10663200DF4D0A0F1B1F22E0C29E20E0020E22E065
:10664200121EF001EB52F64F008311830C2D10E065
:10665200000F111FF801E559F04F208131810C2DF7
:1066620010E0000F111FF801E151F04F2083318338
:1066720002E0C09E00E0000E02E0101EF001EB52AC
:10668200F64F018107FF0EC000E010E022E0C29E3B
:1066920020E0020E22E0121EF001EB52F64F0083C0
:1066A20011831CC002E0C09E00E0000E02E0101E3A
:1066B200F001EB52F64F20813181203004E03007A7
:1066C20068F00FEF13E022E0C29E20E0020E22E00B
:1066D200121EF001EB52F64F0083118390E0FC0191
:1066E200EB56F84FC0828395E7EDFCE0008100FF96
:1066F200C1CD00915F100F3F19F004E1C01649F0BF
:10670200009160100F3F09F4B5CD05E1C01609F004
:10671200B1CD00E890E0FC01EB56F84F0083839581
:1067220000E890E0FC01EB56F84F00838395C9CD59
:10673200282F13E80EEF0E94A54900915E10002356
:1067420021F000E00093DD0CD4C5E2E5F0E1008128
:106752001181E4E5F0E1208131810217130708F489
:10676200C8C500E010E0E2E5F0E100831183CC242B
:1067720027C002E0C09E00E0000E02E0101EF00101
:10678200EB52F64F208131810C2D10E0000F111FCA
:10679200F801E951F14F208331830C2D10E0000FF5
:1067A200111FF801E151F04F208131810C2D10E0D1
:1067B200000F111FF801E355F04F20833183C3947A
:1067C2000FE1C016B0F200915C10002309F09FC0E7
:1067D20001E000935C10E8E5F0E100811181EAE557
:1067E200F0E120813181220F331F021B130BE4E5FC
:1067F200F0E100831183CC2446C00C2D10E0000F81
:10680200111FF801EF5DF14F808191810C2D10E095
:10681200000F111FF801EB55F14F00811181801B10
:10682200910B0C2D10E0000F111FF801E559F04FEC
:1068320000811181212F220F220B322FEAE5F0E194
:106842004081518160E070E00E94954D4CE050E043
:1068520060E070E00E94954D45E050E060E070E03D
:106862000E94DF4D012F122F232F330F330B801B7A
:10687200910B0C2D10E0000F111FF801ED59F14F93
:1068820080839183C3940FE1C01608F0D6C0DD2443
:10689200F601EF5CFF4E0081013009F0AECF0C2D06
:1068A20010E0000F111FF801EF5DF14F008111811F
:1068B2002C2D30E0220F331FF901EB55F14F2081CF
:1068C2003181021B130B212F220F220B322FE4E501
:1068D200F0E14081518160E070E00E94954DE8E571
:1068E200F0E140815181EAE5F0E160817181461B6E
:1068F200570B60E070E00E94DF4D2C2D30E0220F3C
:10690200331FF901ED59F14F00831183BBCF009181
:106912005C100130D1F502E000935C10EAE5F0E191
:1069220000811181E4E5F0E100831183CC240FE1C1
:10693200C01608F082C00C2D10E0000F111FF801E4
:10694200EF5DF14F208131810C2D10E0000F111FFE
:10695200F801ED59F14F00811181201B310B0C2DF3
:1069620010E0000F111FF801EB55F14F008111816A
:10697200201B310B0C2D10E0000F111FF801ED59F7
:10698200F14F20833183C394D2CF00915C10023047
:10699200B1F4E6E5F0E100811181012B61F003E041
:1069A20000935C10E6E5F0E100811181E4E5F0E19D
:1069B2000083118342C000E000935C103EC000914E
:1069C2005C100330D1F5CC2432C002E0C09E00E05E
:1069D200000E02E0101EF001EB52F64F20813181D1
:1069E2000C2D10E0000F111FF801E75DF04F20831E
:1069F200318300E010E02C2D30E0220F331FF9012B
:106A0200E151F04F008311832C2D30E0220F331F10
:106A1200F901EF5DF14F008311832C2D30E0220F3D
:106A2200331FF901E355F04F00831183C3940FE143
:106A3200C01658F200E000935C1000915C10002335
:106A420009F057C4EDE5F0E1008103950083009160
:106A52005D101091AA0C011728F40091E90C002393
:106A620009F4DFC00091E90C002399F5EAEEFCE09D
:106A720000811181ECEEFCE0008311830091A50CF2
:106A8200002329F0E6E9FCE007850A9507870091D3
:106A9200A50C0023F1F40091DB0C013039F400E085
:106AA20010E0EAEEFCE00083118313C00091DB0CDE
:106AB200023041F40091B00C10E0EAEEFCE00083F9
:106AC200118307C00091AF0C10E0EAEEFCE00083F6
:106AD2001183EAEEFCE000811181012B21F401E037
:106AE20000935E109EC000E00093E90CE8EDFCE02C
:106AF20000811181EAEEFCE0208131810217130747
:106B020041F500E010E020E030E0EDE1FEE000833E
:106B12001183228333830091A50C002309F053C013
:106B2200ADE0B0E0A03400E0B00708F04CC0EDE109
:106B3200FEE000811181228133810A0F1B1FF801BF
:106B4200EB52F64F0081FD01EA56F34F0083119696
:106B5200E9CFEAEEFCE00081118120E030E0322F43
:106B6200212F102F00E0110F221F331F005010425F
:106B72002F4F3F4FEDE1FEE00083118322833383E9
:106B82000091A50C0023F9F4ADE0B0E018C0EDE1EE
:106B9200FEE040815181628173818D0120E030E00D
:106BA200040F151F261F371FF801322F3BBF069017
:106BB20000E00BBFFD01EA56F34F00821196A034AC
:106BC20000E0B00720F3EDE1FEE0008111812281B7
:106BD2003381005C1F4F2F4F3F4F0083118322836D
:106BE20033830091AA0C083020F40091AA0C0023F0
:106BF20081F40BE01DE00E94444BEAEEFCE00081D0
:106C020011810E94D20E0DE50E94CB0D01E000938E
:106C12005E100091A50C002309F428CF00E0009338
:106C22005D10A0E0B0E020C0EDE1FEE00081118146
:106C320022813381A801B9014F5F5F4F6F4F7F4FB0
:106C4200EDE1FEE04083518362837383F801322FCA
:106C52003BBF069000E00BBF8D01005C1D4FF801A9
:106C6200EB52F64F00821196A03400E0B00758F5BF
:106C7200E8EDFCE000811181EAEEFCE02081318147
:106C82000217130789F6EDE1FEE0008111812281EE
:106C92003381F801EB52F64F20818D01005C1D4FCC
:106CA200F801EB52F64F2083EDE1FEE00081118105
:106CB200228133810F5F1F4F2F4F3F4F008311837C
:106CC20022833383D0CF00915D100395EAEEFCE07E
:106CD200808191811091AA0C011708F456C000918D
:106CE200DB0C013039F400E010E0EAEEFCE0008356
:106CF200118312C00091A50C023028F0EAEEFCE0EC
:106D02008081918109C00091DB0C023019F48091DD
:106D1200B00C02C08091AF0C90E0E8EDFCE0008185
:106D220011818017910759F400E410E020E030E06F
:106D3200EDE1FEE0008311832283338326C08823A2
:106D420079F4EDE1FEE0008111812281338100546A
:106D5200104020403040008311832283338315C0CA
:106D6200082F10E020E030E0322F212F102F00E01A
:106D7200110F221F331F005C1F412F4F3F4FEDE1C8
:106D8200FEE00083118322833383A0E0B0E01BC0C6
:106D9200EDE1FEE040815181628173818D0120E04D
:106DA20030E0040F151F261F371FF801322F3BBF9B
:106DB200069000E00BBF8D0100581D4FF801EB5209
:106DC200F64F00821196A03400E0B007D0F4E8ED4F
:106DD200FCE0008111818017D9F6EDE1FEE000812F
:106DE2001181228133810A0F1B1FF801EB52F64FEA
:106DF20020818D0100581D4FF801EB52F64F208380
:106E0200E1CF00915E10002309F073C20091530C90
:106E120010E045E00E94644D4091AC0C50E00E94AD
:106E2200704DE6E5F0E1008311830091540C10915E
:106E3200AC0C019F800145E00E946A4DD8010A2FE7
:106E42000B2B11F4A1E0B0E020E030E0CC240EC026
:106E52000C2D10E0000F111FF801EF5DF14F0081C2
:106E620011812017310708F49801C3940FE1C0166D
:106E720008F0F7C0DD24F601E659F64F0081002341
:106E8200A1F30C2D10E0000F111FF801E75DF04F88
:106E92004081518102E0C09E00E0000E02E0101E1F
:106EA200F001EB52F64F408351830C2D10E0000F9E
:106EB200111FF801E951F14F4083518300E010E0C6
:106EC2004C2D50E0440F551FFA01EB55F14F008352
:106ED200118302E0C09E00E4000E02E0101EF001E9
:106EE200EB52F64F008111814C2D50E0440F551F9B
:106EF200FA01EB56F64F60817181DD24F601E4550B
:106F0200F24F4081542F550F550B460F571F040F58
:106F1200151F412F47FF03C000E010E006C00030FC
:106F220044E0140710F00FEF13E04C2D50E0440F33
:106F3200551FFA01E75DF04F40815181B801641B92
:106F4200750B4C2D50E0440F551FFA01EF5DF14FC8
:106F5200608371834C2D50E0440F551FFA01E75DA9
:106F6200F04F608171814C2D50E0440F551FFA01A2
:106F7200E75DF04F0083118342E0C49E40E8040EB7
:106F820042E0141EF001EB52F64F208031804C2D6E
:106F920050E0440F551FFA01EB56F64F0080118066
:106FA200020C131CDD24F601E455F24F4081542FEC
:106FB200550F550B400D511D052E07FE03C040E035
:106FC20050E006C04030E4E05E0710F04FEF53E0BF
:106FD2006017710718F40417150730F00617170722
:106FE20028F44017510710F400E001C001E000232B
:106FF20091F4E6E5F0E100811181012B61F4009149
:107002005D1010E0E091AA0CF0E031970E171F0717
:107012004CF0882339F400E0DD24F601EF5CFF4EEA
:10702200008306C001E0DD24F601EF5CFF4E008321
:107032000C2D10E0000F111FF801EF5DF14F4081A0
:10704200518155230AF004CF0C2D10E0000F111FBF
:10705200F801EF5DF14F008111811195019510400A
:1070620000CF890148E250E00E94544DC8018D01D1
:1070720043E050E00E94544DA8018C010E94704DE3
:10708200E8E5F0E1008311830091AE0C10E0EAE53F
:10709200F0E100831183EAE5F0E100811181000F44
:1070A200111FE8E5F0E12081318102171307E8F1B1
:1070B200E7E6F9E0008102FF13C00BE50E94CB0D69
:1070C20000915D100E94B40D0CE20E94CB0DE8E528
:1070D200F0E1008111810E94D20E0DE50E94CB0DDC
:1070E200E8E5F0E100811181012B39F400E010E0C4
:1070F200EAE5F0E10083118318C0E8E5F0E10081E0
:1071020011810150104016950795EAE5F0E10083E0
:107112001183EAE5F0E100811181012B31F400E0F5
:1071220010E0E8E5F0E100831183E8E5F0E1008199
:10713200118120E030E0000F111F221F331FEAE50A
:10714200F0E180819181A0E0B0E0880F991FAA1F31
:10715200BB1F081B190B2A0B3B0B48015901880C5A
:10716200991CAA1CBB1C880E991EAA1EBB1E000FCE
:10717200111F221F331F088319832A833B83082D83
:1071820009290A290B2929F49924AA24BB24882431
:107192008394088119812A813B81012B022B032BC5
:1071A20041F401E010E020E030E0088319832A83F3
:1071B2003B83CC2442C00419150926093709A401CE
:1071C200B5010E94DF4D2C2D30E0220F331FF90153
:1071D200E559F04F008311830C2D10E0000F111FB1
:1071E200F801E559F04F20813181203004E0300769
:1071F2005CF00FEF13E02C2D30E0220F331FF9016A
:10720200E559F04F008311830C2D10E0000F111F80
:10721200F801E559F04F2081318121300CEF300720
:107222005CF401E01CEF2C2D30E0220F331FF9013A
:10723200E559F04F00831183C3940FE1C01608F0A3
:1072420050C00C2D10E0000F111FF801E355F04F54
:1072520000811181212F220F220B322FAC01BD019F
:107262000E94954D280139010C2D10E0000F111FCD
:10727200F801EF5DF14F00811181212F220F220BC6
:10728200322F0801190140E05AE060E070E080010D
:1072920091010E94954D080119014CE050E060E017
:1072A20070E0800191010E94DF4DDD24F601EF5C68
:1072B200FF4E4081442309F07ECF041915092609A7
:1072C2003709488159816A817B810E94DF4D2C2DCB
:1072D20030E0220F331FF901E559F04F008311838B
:1072E2007BCFEAE5F0E100811181E4E5F0E1008382
:1072F20011832496EEE00C94194E0E94104E402EFB
:107302005524F201E659F64F0081002309F47EC0AC
:1073120002E0409E800100501E4FF801EB52F64FF2
:10732200018105FF06C020E018E1042D0E94034DF3
:107332006DC0E8EDFCE000811181012BC9F002E093
:10734200409E00E0000E02E0101EF001EB52F64FEC
:10735200008111810F7F1370242D30E0220F331F23
:10736200F901EB56F64FA081B181A00FB11F0DC0FC
:1073720002E0409E00E0000E02E0101EF001EB521F
:10738200F64FA081B181AF7FB3700B2F07FF03C00F
:10739200A0E0B0E006C0A03004E0B00710F0AFEF0C
:1073A200B3E014E2042D0E94ED4C0F3F23E01207DC
:1073B20058F4A017B10720F40A1B1B0BC80106C022
:1073C200CD01801B910B02C008E010E096958795D5
:1073D20096958795883000E0900710F488E090E059
:1073E2000EE1009395070A2F00939607AB2FB0E0AA
:1073F200A0939707082F00939807892F90E0809316
:10740200990725E013E0042D0E94204AE6E00C943F
:10741200214E0E94124ED8010091DD0C002309F08A
:1074220041C00A2F0B2BF1F1A03800E0B007D0F5D4
:1074320000E010E0E8EDFCE00083118380E00BC087
:1074420022E0829F900120503E4FF901EB52F64F0D
:107452000083118383958F3110F590E0FC01E6598A
:10746200F64F00810023B1F318E1082F0E94DE4C91
:10747200013029F41EE1082F0E94DD2E04C014E21F
:10748200082F0E94DD2E003020E41207C9F60DED10
:107492001DE00E94444B082F0E94B40DDBCF8D01EA
:1074A2000E941930E4E00C94234E6AC00E94FC0E44
:1074B2001091F40C163018F010E01093F40C209197
:1074C200F40C30E0F901EB50F34F0083E4EFFCE001
:1074D200108113951083053551F50091F40C02507B
:1074E200073008F00A5F10E0F801EB50F34F00811B
:1074F2000F3FE9F400E00093F40C0FEF2091F40C3D
:1075020030E0F901EB50F34F0083E4EFFCE000813F
:107512000395008305E52091F40C30E0F901EB506E
:10752200F34F0083E4EFFCE00081039500830091B8
:10753200F40C063029F50091F50C0F3F09F5009186
:10754200F60C0535E9F40091F70C1091F80C109542
:107552000117B1F40091F90C1091FA0C1095011772
:1075620079F401E00093F30C3091F90C20E00091E2
:10757200F70C10E0020F131FEEEDFCE00083118305
:107582000091FE0C1091FD0C011709F08FCF0895A8
:107592009A938A93C901083C09F0CFC0183151F47B
:1075A200082F092B21F402E00093DB0C01C18C01AE
:1075B20030DFFEC01A3111F01B3149F5E0EEFCE07C
:1075C200808391830FEF0E94CB0D05E50E94CB0DC6
:1075D200E0EEFCE0008111810E94CB0DE0EEFCE0C8
:1075E2000081118100950E94CB0DE0EEFCE000814C
:1075F2001181012F10E00E94CB0DE0EEFCE0008132
:107602001181012F10E000950E94CB0DD1C01F31D6
:1076120059F4882311F401E001C000E0102F10FD9D
:10762200AB9A10FFAB98C4C01232A1F540E050E013
:1076320010E020E030E000E00E94B10C002309F4E9
:10764200B7C0E4EEFCE0008111810817190739F098
:1076520040E050E010E09C0101E00E94B10CE7E53F
:10766200F9E0038114810817190709F4A1C0E7E5BD
:10767200F9E083839483082F23E030E0A9010E947C
:10768200424D892F90E0082F24E030E0A9010E94AA
:10769200424D8EC0113229F4E1EFFCE080839183E8
:1076A20087C0153221F48C010E944C0E81C0163223
:1076B20051F48C010E944C0E0DE00E94CB0D0AE0A9
:1076C2000E94CB0D75C01832A1F540E050E010E0E9
:1076D20020E030E000E00E94B10C002309F468C011
:1076E200E6EEFCE0008111810817190739F0AC01C0
:1076F20010E020E030E004E00E94B10CE7E5F9E0A0
:10770200018512850817190709F452C0E7E5F9E067
:1077120081879287082F29E030E0A9010E94424D1B
:10772200892F90E0082F2AE030E0A9010E94424D03
:107732003FC002E010E8D5D43BC00436F0F00D366D
:10774200E0F42091DD0C222339F021E02093100D8A
:107752002091100D2223E1F7EBE3F7E1212F30E036
:10776200E20FF31F2491223021F49C010E940B4D61
:107772001FC0282F0E94034D1BC02091DD0C222325
:1077820039F021E02093100D2091100D2223E1F712
:10779200E3E0F7E1212F30E0E20FF31F24912230E2
:1077A20021F49C010E940B4D03C0282F0E94034D1F
:1077B200899199910895083C09F0E4C0183181F447
:1077C200EAEEFCE000811181012B29F4ECEEFCE0F1
:1077D200008111810895EAEEFCE000811181089593
:1077E200193121F40091DD0C10E008951A3111F0E5
:1077F2001B3129F4E0EEFCE00081118108951C3177
:1078020011F01D3149F451DE00E00093F30CEEED6E
:10781200FCE00081118108951E3129F446DE0091B9
:10782200F30C10E008951F3141F405B30695069557
:1078320006950095017010E008951232B1F540E00E
:1078420050E010E020E030E000E00E94B10C0023A4
:1078520039F1E7E5F9E003811481E4EEFCE02081EF
:10786200318102171307E1F0E4EEFCE0008111819F
:10787200E7E5F9E003831483E4EEFCE00081118183
:1078820023E030E0A9010E94424DE4EEFCE00081D9
:107892001181012F10E024E030E0A9010E94424D45
:1078A200E7E5F9E0038114810895143269F440E0B8
:1078B20050E010E020E030E000E00E94B10CE2EE87
:1078C200FCE00081118108951032B9F400E0809942
:1078D20002C0006111E00C9902C0086011E00D992C
:1078E20002C0046011E00E9902C0026011E00F991B
:1078F20002C0016011E010E00895113229F4E1EFB5
:10790200FCE00081118108951832B1F540E050E0A9
:1079120010E020E030E000E00E94B10C002339F1D9
:10792200E7E5F9E001851285E6EEFCE02081318190
:1079320002171307E1F0E6EEFCE000811181E7E5B2
:10794200F9E001871287E6EEFCE00081118129E06F
:1079520030E0A9010E94424DE6EEFCE00081118177
:10796200012F10E02AE030E0A9010E94424DE7E534
:10797200F9E001851285089501E010E8B2D30FEF16
:107982001FEF08950436E8F00E36D8F42091DD0C8E
:10799200222339F021E02093100D2091100D222393
:1079A200E1F7EBE3F7E1212F30E0E20FF31F24913F
:1079B200223019F40E94ED4C08950E94DE4C10E032
:1079C20008950F31D8F42091DD0C222339F021E003
:1079D2002093100D2091100D2223E1F7E3E0F7E14F
:1079E200212F30E0E20FF31F2491223019F40E947C
:1079F200ED4C08950E94DE4C10E0089500E010E086
:107A020008959A938A93E1E1FDE000811181980142
:107A12002F5F3F4FE1E1FDE02083318320E030E042
:107A2200005010462F4F3F4FF801322F3BBF0690B8
:107A3200002D10E01BBFE1E1FDE0408151819A0180
:107A42002F5F3F4FE1E1FDE02083318360E070E092
:107A5200405050466F4F7F4FFA01362F3BBF069082
:107A6200202D10E01BBFE1E1FDE040815181CA0100
:107A72000196E1E1FDE08083918360E070E0405097
:107A820050466F4F7F4FFA01362F3BBF069010E0F2
:107A92001BBF002321F4102D022F8DDE4EC00230B9
:107AA20061F4102D30E0220F331FF901E35EF24F33
:107AB20020813181022F7FDE40C0013069F4002D28
:107AC20010E0000F111FF801E35EF24F00811181F7
:107AD200102F022F70DE31C00330A9F4002D10E008
:107AE200000F111FF801E35EF24F00811181102F88
:107AF20030E0220F331FF901E35EF24F2081318122
:107B0200022F59DE1AC0043039F4502D40E0022F02
:107B120010E0040F151F11C0053069F4102D00E0AC
:107B220030E0200F311F220F331FF901E35EF24FC5
:107B32000081118102C000E010E0899199910895BD
:107B42000E94124EA801E1E1FDE00081118198013D
:107B52002F5F3F4FE1E1FDE02083318320E030E001
:107B6200005010462F4F3F4FF801322F3BBF069077
:107B7200002D10E01BBFE1E1FDE000801180C0019B
:107B82000196E1E1FDE080839183C001A0E0B0E0D5
:107B920080509046AF4FBF4FFC013A2F3BBF06903B
:107BA200602D10E01BBFE1E1FDE000801180C0010B
:107BB2000196E1E1FDE080839183C001A0E0B0E0A5
:107BC20080509046AF4FBF4FFC013A2F3BBF06900B
:107BD20010E01BBF002329F49A01102D062FD8DCD8
:107BE2004BC0023069F49A01102D70E0660F771FC6
:107BF200FB01E35EF24F40815181042FC9DC3CC09E
:107C0200013071F49A01002D10E0000F111FF801EC
:107C1200E35EF24F00811181102F062FB9DC2CC0D8
:107C22000330B1F49A01002D10E0000F111FF8018A
:107C3200E35EF24F00811181102F70E0660F771F13
:107C4200FB01E35EF24F40815181042FA1DC14C09D
:107C5200043021F407E010E044D20EC0053061F494
:107C6200102D00E070E0600F711F660F771FFB019F
:107C7200E35EF24F40835183E4E00C94234EC1DE75
:107C8200E3E1FDE000831183E1E1FDE00081118188
:107C920098012F5F3F4FE1E1FDE02083318320E037
:107CA20030E0005010462F4F3F4FF801322F3BBFBC
:107CB200069000E00BBF0092190DA3DEE5E1FDE0A6
:107CC200008311830091190D002379F4E3E1FDE0B3
:107CD20000811181E5E1FDE0208131810217130766
:107CE20011F401E0089500E008950091190D0130AA
:107CF20079F4E5E1FDE000811181E3E1FDE020811D
:107D020031810217130710F401E0089500E008958D
:107D12000091190D023079F4E3E1FDE00081118157
:107D2200E5E1FDE0208131810217130710F001E047
:107D3200089500E008950091190D033079F4E3E10C
:107D4200FDE000811181E5E1FDE020813181021732
:107D5200130710F401E0089500E008950091190D51
:107D6200043079F4E5E1FDE000811181E3E1FDE019
:107D7200208131810217130710F001E0089500E01D
:107D820008950091190D053079F4E3E1FDE00081D9
:107D92001181E5E1FDE0208131810217130711F025
:107DA20001E0089500E0089505E010E09AD100E0B6
:107DB200089500911A0D013061F400911C0D002309
:107DC20031F000911B0D002311F001E0089500E055
:107DD200089500911A0D023061F400911C0D0023E8
:107DE20021F400911B0D002311F001E0089500E041
:107DF200089506E010E075D100E008959A938A9301
:107E02000230C9F0E1E1FDE0408151819A012F5F2A
:107E12003F4FE1E1FDE02083318360E070E04050BC
:107E220050466F4F7F4FFA01362F3BBF069010E04E
:107E32001BBF0092180D1091180D1F5F09F440C16D
:107E4200125091F01A9509F11A9509F44CC01A953D
:107E520009F4F2C01A9509F4FBC01A9509F407C196
:107E62001A9509F41CC137C1002331F0CADDE1E1E2
:107E7200FDE00083118332C1E1E1FDE00081118167
:107E82000D5F1F4F0083118329C1002319F1E1E126
:107E9200FDE0008111810D5F1F4F00831183B1DD71
:107EA200E5E1FDE000831183E1E1FDE00081118164
:107EB2000650104000831183E5E1FDE0008111814D
:107EC2003FDEE1E1FDE0008111810D5F1F4F008384
:107ED200118304C1E1E1FDE0008111810A5F1F4FBE
:107EE20000831183FBC0002309F49DC0E1E1FDE0A2
:107EF200008111810D5F1F4F0083118382DDE3E159
:107F0200FDE000831183E1E1FDE000811181980130
:107F12002F5F3F4FE1E1FDE02083318320E030E03D
:107F2200005010462F4F3F4FF801322F3BBF0690B3
:107F320000E00BBF0092190D64DDE5E1FDE0008376
:107F420011830091190D002359F4E3E1FDE0008152
:107F52001181E5E1FDE080819181800F911F50C088
:107F62000091190D013059F4E3E1FDE08081918126
:107F7200E5E1FDE000811181801B910B41C0009180
:107F8200190D023061F4E3E1FDE000811181E5E1C8
:107F9200FDE0408151810E94544DC80131C00091E1
:107FA200190D033061F4E3E1FDE000811181E5E1A7
:107FB200FDE0408151810E94704DC80121C00091B5
:107FC200190D003159F4E3E1FDE000811181E5E191
:107FD200FDE0808191818023912312C00091190DCF
:107FE200013159F4E3E1FDE000811181E5E1FDE0B9
:107FF20080819181802B912B03C004E010E071D02D
:10800200E1E1FDE0008111810A50104000831183FB
:108012008C0196DDE1E1FDE000811181095F1F4FD6
:10802200008311835BC0E1E1FDE000811181065F05
:108032001F4F0083118352C0002309F04FC0E1E1BA
:10804200FDE000811181E1E1FDE00083118346C082
:10805200002321F00BE10093170D40C0E1E1FDE0A8
:1080620000811181E1E1FDE00083118337C000232B
:1080720069F0E1E1FDE0008111810D5F1F4F61D2E6
:10808200C0DCE1E1FDE00083118328C0E1E1FDE015
:10809200008111810D5F1F4F008311831FC00023D8
:1080A20031F079D2E1E1FDE00083118317C0E1E113
:1080B200FDE000811181E1E1FDE0008311830EC04A
:1080C200002361F4E1E1FDE000811181E1E1FDE0E5
:1080D2000083118303C003E110E003D089919991D9
:1080E20008959A938A93C801E7E6F9E0008101FFB7
:1080F2001AC00AE515E10E94444B8C010E94D20E7F
:108102000BE50E94CB0DE1E1FDE0008111810E94AF
:10811200D20E0AE30E94CB0D0091180D0E94B40DFD
:108122000DE50E94CB0D8991999108950E94134EFD
:10813200A02FAA2311F49598969A00E010E0E1E1AD
:10814200FDE00083118380E090E204E00093180DCB
:10815200AA2321F00BE115E10E94444B00E00093B9
:10816200170D05C002E04ADEAA2309F013D10091DF
:10817200170D0B3109F407C1E1E1FDE020813181E6
:10818200203000EC300708F0FEC00091180D0530D9
:1081920009F4F9C0E1E1FDE0008111810817190736
:1081A20008F0F1C0E1E1FDE00081118198012F5F4B
:1081B2003F4FE1E1FDE02083318320E030E00050D9
:1081C20010462F4F3F4FF801322F3BBF069000E081
:1081D2000BBF0092180DE8E1FDE0008107FFC2CF5E
:1081E2000091180D005849F00A9509F46FC00A95DC
:1081F20009F4B0C00A95B1F1C2C041DD00931B0D74
:1082020000911B0D00931C0DE1E1FDE00081118145
:1082120098012F5F3F4FE1E1FDE02083318320E0B1
:1082220030E0005010462F4F3F4FF801322F3BBF36
:10823200069000E00BBF00921A0DAA2309F0AAD003
:1082420000911A0D002309F092CF00911C0DD6DD8A
:10825200AA2309F48CCF00911C0D002309F487CFC7
:1082620099D085CF0CDD00931B0DA3DD00931C0D6F
:10827200E1E1FDE00081118198012F5F3F4FE1E1D3
:10828200FDE02083318320E030E0005010462F4F84
:108292003F4FF801322F3BBF069000E00BBF009228
:1082A2001A0DAA2309F076D000911A0D002309F0C5
:1082B2005ECF00911C0DA2DDAA2309F458CF0091D4
:1082C2001C0D002309F453CF65D051CF00911C0D32
:1082D200002359F0E1E1FDE000811181085F1F4FA9
:1082E2000083118300E08ADD42CFC9DC00931B0DBD
:1082F20000911B0D00931C0DE1E1FDE00081118155
:1083020098012F5F3F4FE1E1FDE02083318320E0C0
:1083120030E0005010462F4F3F4FF801322F3BBF45
:10832200069000E00BBF00921A0DAA2309F032D08A
:1083320000911A0D002309F01ACF00911C0D5EDD89
:10834200AA2309F414CF00911C0D002309F40FCFC6
:1083520021D00DCFAA2309F01DD000911C0D0023BE
:1083620011F401E001C000E049DDAA2309F4FFCEC7
:1083720000911C0D002309F0FACE0CD0F8CE00E1DA
:1083820010E0AFDEF4CE0091DD0C0023E1F7E3E074
:108392000C94244E0CE810E00E94444B66D00DE28F
:1083A2000E94CB0D0091180D0E94B40D0AE30E94A9
:1083B200CB0D00E20E94CB0D00911B0D0E94B40D6B
:1083C2000DE30E94CB0D08E20E94CB0DE3E1FDE03C
:1083D200008111810E94D20E0CE20E94CB0D00E2BC
:1083E2000E94CB0D0091190D0E94B40D0CE20E9467
:1083F200CB0D00E20E94CB0DE5E1FDE00081118191
:108402000E94D20E09E20E94CB0D00E20E94CB0D27
:1084120000911A0D0E94B40D0BE70E94CB0D009142
:108422001C0D0E94B40D0DE70E94CB0D0BE50E94BE
:10843200CB0DE1E1FDE0008111810E94D20E0DE53C
:108442000E94CB0D0E94FC0E0093170D0091170D98
:108452000B3151F40DE415E10E94444BE1E1FDE0E2
:10846200008111810E94D20E08950091180D0038EA
:1084720029F404E615E10E94444B08950091180D79
:10848200013829F40CE615E10E94444B089500914D
:10849200180D023829F404E715E10E94444B0895AF
:1084A2000091180D033829F40CE715E10E94444BA2
:1084B20008950091180D013029F404E815E10E9495
:1084C200444B08950091180D023029F40CE815E18F
:1084D2000E94444B08950091180D033029F404E9D9
:1084E20015E10E94444B08950091180D043029F4BF
:1084F2000CE915E10E94444B08950091180D0530D6
:1085020029F404EA15E10E94444B08950091180DE4
:10851200063029F40CEA15E10E94444B08950091BB
:10852200180D073029F404EB15E10E94444B08951D
:108532000091180D0F3F21F40CEB15E10E94444B02
:1085420008952091AB0D2A3010F52091AB0D30E04B
:10855200220F331FF901EF57F24F00831183EBEA29
:10856200FDE000810395008320911C0D30E0009115
:10857200AB0D10E0000F111FF801EF57F24F2083EF
:108582003183EBEAFDE0008103950083089509E061
:1085920010E0A7DD08950091AB0D0023E9F0EBEAAE
:1085A200FDE000810A95008310E0000F111FF80121
:1085B200EF57F24F0081118100931C0DEBEAFDE0B1
:1085C20000810A95008310E0000F111FF801EF5798
:1085D200F24F0081118108950AE010E082DD0FEF71
:1085E2001FEF08950E94124E00916110002309F0BE
:1085F200D3C000915E09013009F094C0E4EDFDE0C2
:1086020002811381012B09F45AC000E00093CB0DC3
:1086120000E010E0E0EDFDE00083118300E010E0F7
:10862200E2E6F0E10083118301E000936110E4EDE2
:10863200FDE00081118145E050E00E94704D10E0A4
:10864200ECECFDE000831183ECECFDE08081918194
:10865200E4EDFDE00281138145E050E00E94704D9F
:1086620010E0801B910BEEECFDE080839183EEEC39
:10867200FDE020813181243700E0300720F003E063
:108682000093DD0D27C2EEECFDE02081318122371F
:1086920000E0300720F007E00093DD0D1BC2EEEC96
:1086A200FDE020813181203700E0300720F00FE02B
:1086B2000093DD0D0FC20FE00093DD0D0BC20091A0
:1086C200CB0D0370002309F005C2E4EDFDE000814B
:1086D200118145E050E00E94704D10E0ECECFDE0AD
:1086E20000831183ECECFDE080819181E4EDFDE0FB
:1086F2000281138145E050E00E94704D10E0801B22
:10870200910BEEECFDE080839183EEECFDE02081A5
:108712003181293500E0300708F0DCC10FE7009312
:10872200DD0DD8C1E4EDFDE002811381012B09F0DA
:10873200D1C10091CB0D0370002309F0CBC1E4ED50
:10874200FDE00081118145E050E00E94704D10E093
:10875200ECECFDE000831183ECECFDE08081918183
:10876200E4EDFDE00281138145E050E00E94704D8E
:1087720010E0801B910BEEECFDE080839183EEEC28
:10878200FDE020813181293500E0300708F0A2C1E7
:108792000FE70093DD0D9EC100916110013009F0D9
:1087A2004AC1E4EDFDE002811381012B61F400E096
:1087B20010E01BBD0ABD00E00093DD0DA89800E0AB
:1087C2000093611087C10091CB0D0F71002329F432
:1087D20000E010E01BBD0ABD7DC10091CB0D0F7101
:1087E200023009F077C1E4EDFDE00081118145E03E
:1087F20050E00E94704D10E0ECECFDE0008311832C
:10880200ECECFDE080819181E4EDFDE002811381D9
:1088120045E050E00E94704D10E0801B910BEEECA1
:10882200FDE080839183E0EDFDE000811181EEECBB
:10883200FDE0208131810217130740F4EEECFDE0E8
:1088420000811181E0EDFDE000831183E3E0F6E1B8
:10885200A8EDBDE00D911C911197169507951695FF
:108862000795E00FF11F049110E0E2EDFDE00083B7
:108872001183EEECFDE0008111810A5F1F4FECECE9
:10888200FDE0208131810217130718F00FEF13E08A
:1088920010C00AEF17E1ECECFDE040815181EEECF3
:1088A200FDE020813181421B530B465050400E9413
:1088B200704D003024E0120710F00FEF13E01BBDE3
:1088C2000ABDA2EDBDE0ED91FC911197F69720F063
:1088D20003E00093DD0D32C0A2EDBDE0ED91FC910D
:1088E2001197F49720F007E00093DD0D27C0EEEC1E
:1088F200FDE020813181243700E0300720F003E0E1
:108902000093DD0D1BC0EEECFDE0208131812237AA
:1089120000E0300720F007E00093DD0D0FC0EEEC21
:10892200FDE020813181203700E0300720F00FE0A8
:108932000093DD0D03C00FE00093DD0DE2E6F0E1F0
:10894200008111810F5F1F4F00831183E2E6F0E186
:1089520020813181283601E0300758F000E010E034
:108962001BBD0ABD0FEF0093DD0D02E800936110FD
:10897200B1C0EEECFDE020813181263700E0300706
:1089820058F000E010E01BBD0ABD0FEF0093DD0DB3
:1089920001E8009361109EC0E0EDFDE000811181CD
:1089A2000C531040EEECFDE02081318102171307D9
:1089B20098F0EEECFDE020813181253600E03007B1
:1089C20058F000E010E01BBD0ABD0FEF0093DD0D73
:1089D20003E8009361107EC0E2EDFDE02081318169
:1089E2002C3300E0300758F000E010E01BBD0ABD58
:1089F2000FEF0093DD0D04E8009361106BC0A2ED50
:108A0200BDE0ED91FC911197F89708F463C0EEEC8C
:108A1200FDE020813181203700E0300708F45AC0A0
:108A220000E010E01BBD0ABD0FEF0093DD0D04E86E
:108A3200009361104FC000915E09023041F002E0E4
:108A420000935E0927E030E0A9010E94424DE4ED67
:108A5200FDE002811381012BC1F400E010E01BBD97
:108A62000ABD00E00093DD0DA89800E000936110BC
:108A720000915E09002371F100E000935E0927E096
:108A820030E0A9010E94424D25C00091CB0D0F712B
:108A9200002301F5E4EDFDE00081118145E050E0A5
:108AA2000E94704D10E0ECECFDE000831183ECECD1
:108AB200FDE080819181E4EDFDE00281138145E0DA
:108AC20050E00E94704D10E0801B910BEEECFDE037
:108AD20080839183E4E00C94234E07EE06B900E014
:108AE20010E01BBD0ABD03EC0FBD02E00EBD03E0AA
:108AF2000093DC0DECEDFDE0008103950083037033
:108B020007B901E010E00E945C0C24B135B100917C
:108B1200DC0D10E003701070000F111FF801EC5211
:108B2200F24F20833183ECEDFDE000810395008359
:108B3200037007B901E010E00E945C0C24B135B16A
:108B42000091DC0D10E003701070000F111FF8018E
:108B5200EC52F24F20833183ECEDFDE0008103956E
:108B62000083037007B901E010E00E945C0C24B19D
:108B720035B10091DC0D10E003701070000F111F71
:108B8200F801EC52F24F20833183ECEDFDE00081DD
:108B920003950083037007B901E010E00E945C0CAA
:108BA20024B135B10091DC0D10E003701070000F9C
:108BB200111FF801EC52F24F2083318308950E9475
:108BC200134E1A981B9A0E94D80BA89800E00093A3
:108BD20065090093660900E000936709009368093C
:108BE20000E00093DD0C00E00093EE0C22E030E0A8
:108BF200A9010E94364D0F3FA9F021E030E0A90102
:108C02000E94364D0F3F71F023EF3FE0A9010E9411
:108C1200364D033038F427E030E0A9010E94364D8A
:108C2200033048F101E00093580921E030E0A90146
:108C32000E94424D02E20093570920E030E0A90170
:108C42000E94424D00E022E030E0A9010E94424D24
:108C520080E023EF3FE0082FA9010E94424D0AE085
:108C62000093EE0C00E000935E0927E030E0A901DA
:108C72000E94424D37C021E030E0A9010E94364DEA
:108C82000093580920E030E0A9010E94364D00937C
:108C9200570923EF3FE0A9010E94364D802F23E0C0
:108CA20030E0A9010E94364D00935A0924E030E0D9
:108CB200A9010E94364D00935B0929E030E0A90129
:108CC2000E94364D009360092AE030E0A9010E941B
:108CD200364D0093610927E030E0A9010E94364D2C
:108CE20000935E0900E000935F0911E020E830E0A4
:108CF20000E00E94B90B21E01091570900E00E94A8
:108D0200280C21E012E201E00E94280C00E000930E
:108D1200650900936609E1DE789424EF3FE0A9013A
:108D22000E94364D053519F400E0C8D45EC1833087
:108D320038F080E023EF3FE0082FA9010E94424D66
:108D420094B700E004BF21EF3FE0A9010E94364D35
:108D5200002361F0923051F48395833008F080E073
:108D620023EF3FE0082FA9010E94424D9A709923F8
:108D720061F400915E09002341F000E000935E0976
:108D820027E030E0A9010E94424D21EF3FE0A90116
:108D92000E94364D013031F001E021EF3FE0A901A0
:108DA2000E94424D00915E09023009F05DC000E868
:108DB200009361100FEF0093DD0D56C090E0809B91
:108DC20004C002E310E00E945C0C0091FE0C1091C2
:108DD200FD0C011769F00E94FC0EA02FA53521F4AD
:108DE2000091FD0C0093FE0C082F0E94CB0D01C0D8
:108DF200A0E0882311F4AC9807C0813011F4AD983B
:108E020003C0823009F4AE98933209F046C0A3320F
:108E120009F043C004E110E00E945C0C08E001BDCF
:108E2200809B04C002E310E00E945C0C0C991CC001
:108E320002E310E00E945C0C00915E09002371F4D1
:108E4200E4EDFDE002811381012B41F001E000938A
:108E52005E0927E030E0A9010E94424D0C9BFECF43
:108E620002E310E00E945C0C809B31C0AD9AAC9A88
:108E7200AE9A0091FE0C1091FD0C011709F49ECFE1
:108E82000E94FC0E902F953521F40091FD0C009369
:108E9200FE0C082F0E94CB0D92CF993011F0A93011
:108EA20089F404E110E00E945C0C08E001BD8395A6
:108EB200833008F080E023EF3FE0082FA9010E94F1
:108EC200424DAECF9D3019F0AD3009F0A9CF21EF60
:108ED2003FE0A9010E94364D002331F000E021EF6E
:108EE2003FE0A9010E94424D809BFECF04E110E0C9
:108EF2000E945C0C00E910E0C6D38ED3882391F463
:108F020001E0DCD3902F0CE810E0BDD3092F0E94C2
:108F1200100F08E512E0B7D301E0009367090E9441
:108F2200200FFDCF00915709013059F101E0009364
:108F320057092091570914E00EEF64D505E912E0B4
:108F4200A2D300E814E82EE130E04091570950E046
:108F520060E070E04F5F5F4F6F4F7F4F0E94DF4DC9
:108F62000E94F30D00EB12E08ED30091570920E02E
:108F720030E0A9010E94424D09B904EF11E00E94BC
:108F82005C0C01E010E0E8EDFCE00083118301E0FD
:108F920095D3902F0CE810E076D3092F0E94100F82
:108FA20008E512E070D307E0009367090E944E21A2
:108FB200E4EDFDE020813181273302E0300730F01B
:108FC20023E333E012E20EEF25D505C02FEF33E0A5
:108FD20012E20EEF1FD5813071F401E010E0E8EDEE
:108FE200FCE0008311830E946B2203E00093670977
:108FF2000E94DF2316C08230A1F404E610E00E9432
:109002005C0C02E00093670900E00E94974004E6CE
:1090120010E00E945C0C04E110E00E945C0C08E08D
:1090220001BDFFCFFA93EA934A933A932A931A9394
:109032000A933FB74BB700E00BBFAA9820919C0060
:109042000091FD0C10E00F701070F801E150F34F29
:109052002083EDEFFCE00081039500834BBF3FBF0F
:1090620009911991299139914991E991F9911895AB
:10907200FA93EA934A933A932A931A930A933FB73D
:109082004BB700E00BBF00916509102F13951093A9
:1090920065092CB110E0F801EB56F94F20834BBF64
:1090A2003FBF09911991299139914991E991F9911A
:1090B20018952497AA98A99808EA10E0E4D223C048
:1090C2000E94FC0E0E94C70D5E9A0091FE0C109148
:1090D200FD0C0117A9F75E9BFECF1A981B9A00910F
:1090E200660910916509011771F00091660910E097
:1090F200F801EB56F94F0081E6E6F9E0108113958D
:1091020010830E94CB0D0091FE0C1091FD0C0117F3
:1091120031F31B981A9AD9CF0E940F4EAA98A99898
:1091220008EA10E0B0D218C05E9BFECF1A981B9AD4
:109132000091660910916509011771F000916609A5
:1091420010E0F801EB56F94F0081E6E6F9E01081F4
:10915200139510830E94CB0D0091FE0C1091FD0C13
:10916200011731F31B981A9A1CC0FC013A2F3BBF1E
:109172000690002D10E01BBF8F5F9F4FAF4FBF4F78
:10918200600E0E94C70D5E9A01E0400E00E0501E84
:109192000FEF401607E1500640F3062D0E94C70D5F
:1091A2005E9A0091FE0C1091FD0C011709F4BCCFE0
:1091B2000E94FC0E0E3741F480E090ECA0E0B0E09B
:1091C200662444245524E4CF0E94C70D5E9AE9CF59
:1091D2000E94114E902F44249F3F29F400E014EF87
:1091E20021E030E004C008EE13E020E030E080E04F
:1091F20013C04091660950E0FA01EB56F94F4081E5
:10920200E6E6F9E0508153955083682F70E0FB0148
:10921200E95EF74F408383958917D8F440E050E028
:1092220060E070E00090660910906509011479F41D
:109232000A011B01A001B1014F5F5F4F6F4F7F4FCA
:10924200001511052205330568F744244394442090
:1092520081F2A82FB0E00091CD080E3F09F470C052
:10926200442071F09F3F61F0E7E6F9E0008100FFE2
:1092720003C00FE11DE007D2009165090093660962
:10928200A43008F45DC0009117080F3F21F400914B
:1092920018080F3F71F0E7E6F9E0008100FF03C014
:1092A20004E31DE0F0D1009165090093660900E036
:1092B20048C0009119081091CD08011771F0E7E636
:1092C200F9E0008100FF03C00AE41DE0DCD1009157
:1092D20065090093660900E034C020911A0830E065
:1092E2000A2F10E0045010402017310771F0E7E612
:1092F200F9E0008100FF03C000E61DE0C4D1009147
:1093020065090093660900E01CC082E007C090E096
:10931200FC01E95EF74F0081B00F83958A17B8F31D
:10932200BF3F71F0E7E6F9E0008100FF03C006E706
:109332001DE0A9D1009165090093660900E001C012
:109342000A2FE5E00C94224E0E94124E3FEF30931A
:10935200CB083FEF3093CC080093CD08022F0E5F6D
:109362000093CE081093CF0880E00DC090E0FC017E
:10937200EB56F84F0081A82FB0E01596FD01E5539A
:10938200F74F00838395821788F300E02A5FA22FAC
:1093920082E007C090E0FC01E553F74F1081010F16
:1093A200839590E0EA2FF0E031978E179F0794F3B0
:1093B200009590E0FC01E553F74F00831B981A9A41
:1093C20080E009C05E9A90E0FC01E553F74F00810E
:1093D2000E94C70D83958A17A8F35E9BFECF1A9849
:1093E2001B9A0A2FE4E00C94234E0E94124ED801DD
:1093F200922F992359F40091CD080E3F21F400EFEA
:1094020011E041D103C001E112E03DD180E00CC086
:10941200082F10E0FD01E00FF11F00810E94830E72
:1094220000E20E94CB0D8395891790F301E412E0CC
:109432002AD1092F0E94100FE4E00C94234E0E94BF
:10944200104E802F912F422E01E00093DC0CB0E0F1
:109452002DC040E050E060E070E0F0E08A019B0146
:10946200A801B9014F5F5F4F6F4F7F4F083EE3E0A6
:109472001E07E0E02E07E0E03E0798F4009166093F
:1094820010916509011751F300916509009366096E
:1094920040E050E060E070E00F2FF02FF3950536CA
:1094A200E8F20091650900936609B395B23008F0BD
:1094B20051C00091650900936609242D192F082FC8
:1094C20043DFA02F913061F48E3F29F455245A9442
:1094D2005092690930C006E0502E509269092BC0A3
:1094E200923039F45090960706E0500E5092690976
:1094F20022C08E3FC1F08F3140F4082F10E0F801F6
:10950200E659F64F0081023870F0843680F08E36CC
:1095120070F4082F10E004561040F801E657F64F99
:109522000081023820F455245092690913C006E0E4
:10953200502E50926909552009F4B7CF052D48DE07
:109542000093690900916909051521F00FEF501682
:1095520009F07FCF00E00093DC0C0091690905154A
:1095620009F443C00091CD080E3FF9F1E7E6F9E0B6
:10957200008100FF15C00DED1DE085D0082F0E946F
:10958200100F07EB10E07FD02A2F0BEC18E02DDF35
:1095920009EC10E078D02091690907E118E025DF95
:1095A200E7E6F9E0008101FF1EC000E011E80E9439
:1095B2007240082F0E94830E00E20E94CB0D092FF9
:1095C2000E94830E00E20E94CB0D009195070E943B
:1095D200830E00E20E94CB0D009196070E94830E3B
:1095E20000E20E94CB0D00E014C000916809002344
:1095F20079F007EB10E047D02A2F0BEC18E0F5DEEC
:1096020009EC10E040D02091690907E118E0EDDE95
:1096120001E0E6E00C94214E0BED10E034D000E8BE
:1096220014E82EE130E04091990050E060E070E0F3
:109632004F5F5F4F6F4F7F4F0E94DF4D0E94F30DD0
:1096420000E20E94CB0D00EB12E01DD00CE20E9462
:10965200CB0D05EE10E017D000E814E82EE130E063
:1096620049B150E060E070E04F5F5F4F6F4F7F4F56
:109672000E94DF4D0E94F30D00E20E94CB0D00EB31
:1096820012E001D00895EF97EF97A49720E001C070
:109692002395203A60F430E0F801E20FF31F449181
:1096A200FE0130E0E20FF31F4083442389F78E016D
:1096B2000E94EF0EEF96EF96A49608950E94124E26
:1096C200B02FBB2361F00CE810E0DDDF09E40E945B
:1096D200CB0D04E40E94CB0D0AE30E94CB0D90E077
:1096E20020E011E00EEFABDE00916909002309F4DE
:1096F20094C0A0E00EC0843658F08E3648F420E0C4
:10970200082F10E004561040F801E657F64F208368
:10971200A39500916909A01708F07FC00A2F10E0F5
:10972200F801E95EF74F00810F3F91F70A2F10E031
:109732000F5F1F4FF801E95EF74F00810F3F41F7BE
:109742000A2F10E00E5F1F4FF801E95EF74F80818C
:109752000A2F10E00D5F1F4FF801E95EF74F0081FD
:10976200023009F04FC00A2F10E00E5F1F4FF801C0
:10977200E95EF74F208130E00A2F10E00D5F1F4FA6
:10978200F801E95EF74F408150E0420F531F0A2F64
:1097920010E00C5F1F4FF801E95EF74F208130E0C7
:1097A200240F351F0A2F10E00B5F1F4FF801E95EEF
:1097B200F74F008110E0020F131F0F3F20E0120746
:1097C20009F58F3140F420E8082F10E0F801E6593E
:1097D200F64F20830DC0843658F08E3648F420E8C8
:1097E200082F10E004561040F801E657F64F208388
:1097F200BB2331F0082F0E94830E00E20E94CB0DA2
:10980200939586CF8F3108F076CF20E0082F10E0B5
:10981200F801E659F64F20837BCF40EC50EE60E032
:1098220070E080E059C002E0809F8001212F220F6A
:10983200220B322F040F151F261F371F0F5F1F4FDA
:109842002F4F3F4FF801322F3BBF0690102D00E003
:109852000BBF00E022E0829F212C220C2208322C36
:10986200040E151E261E371EF001322D3BBF069038
:1098720020E02BBF1124000E111E082F10E0000F54
:10988200111FF801EB56F64F00821182082F10E0EB
:10989200000F111FF801EB56F64F20813181203065
:1098A20000E4300769F0082F10E0000F111FF801E3
:1098B200EB56F64F20813181203000E4300759F415
:1098C20000E010E0282F30E0220F331FF901EB56A1
:1098D200F64F0083118383958F3108F4A4CF80E083
:1098E20012C014E2082F0E94DD2E0060106222E0F6
:1098F200829F20E0020E22E0121EF001EB52F64F90
:109902000083118383958F3180F5082F10E0F801D1
:10991200E659F64F00810023A9F310E1082F4DD03C
:109922000068282F30E0F901E659F64F008315E070
:10993200082F43D0002321F020E015E0082F62D049
:1099420018E1082F3AD0013061F61EE1082F0E947B
:10995200DD2E22E0829F20E0020E22E0121EF001A4
:10996200EB52F64F00831183CDCF84E620C0A82F9F
:10997200B0E0A456B040FD01E657F64F0081002347
:10998200A9F010E1082F19D00068A82FB0E0A45662
:10999200B040FD01E657F64F008315E0082F0DD0C9
:1099A200002321F020E015E0082F2CD083958E367D
:1099B200F0F2092FE4E00C94234E1093950711E086
:1099C2001093960722E012E03ADD002319F000918D
:1099D2001C0808950FEF08951093950712E0109355
:1099E200960722E012E02BDD002349F030911D089A
:1099F20020E000911C0810E0020F131F08950FEFE2
:109A02001FEF0895109395072093960722E013E025
:109A120016DD089510939507122F10939607232FA2
:109A220030E02093970723E013E009DD08950FE368
:109A32000DBF05E00EBFC0E0D5E00E942E4E002310
:109A420011F00E94404E00E00BBF0E94E0450E94D0
:109A5200634E0C94634EE199FECF08954F5F5F4FC2
:109A6200FADF4EBB5FBBE09A0895FADF0DB30895AB
:109A72004F5F5F4F4EBB5FBBF894E29AE19A0FBE15
:109A820008950FB6E8DF0DBBF5CF0024E8E0EA95B4
:109A920032F0001F001C0416D0F3041AF8CF001F86
:109AA200402D00950895002411240030010741F053
:109AB2001695079510F4040E151E440F551FF5CF89
:109AC200002D112D08954A951AF0000F111FFBCF9A
:109AD20008954A951AF016950795FBCF089500242C
:109AE2001124EFE0001F111F001C111C04161506A3
:109AF20010F0041A150AEA95AAF7001F111F402D4B
:109B0200512D009510950895309520951095019549
:109B12001F4F2F4F3F4F0895709560955095419577
:109B22005F4F6F4F7F4F0895002411242224332466
:109B3200E02FE12BE22BE32B71F036952795179559
:109B4200079520F4040E151E261E371E440F551FBE
:109B5200661F771FEDCF002D112D222D332D089575
:109B62004A952AF0000F111F221F331FF9CF0895C3
:109B72000024112422243324E0E2EA9592F0001F0B
:109B8200111F221F331F001C111C221C331C041620
:109B920015062606370688F3041A150A260A370A16
:109BA200ECCF001F111F221F331F402D512D622D9C
:109BB200732D00951095209530950895FF277723F2
:109BC2001AF4F1600E948D4D33231AF4F0950E942D
:109BD200854D0E94B94DF69510F40E94854DF6957B
:109BE20010F40C948D4D0895AF93BF93B12FA02F15
:109BF2003BBFD895EF5FFF4F3F4F0D924150504012
:109C0200B9F74BBFBF91AF910895FA92EA92DA92F7
:109C1200CA92BA92AA929A928A927A926A925A9222
:109C22004A92BA93AA939A938A930895FF84EE84F0
:109C3200DD84CC84BB84AA84998488847F806E80EE
:109C42005D804C80BB81AA8199818881F0E00FB64A
:109C5200F894CE0FDF1F0FBE089501E0089520E0B3
:109C620002D0E9F708952D9301501040202F212BA7
:109C720008953BBF27913BB7F6DFD9F7089507E177
:109C82001DE92801F20130E03BBF07911691F20174
:109C92003296A791B691F201349647915791669107
:109CA200242F252B262B21F0FA01362FE2DF01C0CB
:109CB200D6DF07E0400E00E0501EA20145325D49AA
:109CC20008F3089500008895FECF141A1F24292E48
:109CD20033383D4D151B20252A2F34390808080931
:109CE20009090909090909090909090909090909E2
:109CF2000808080808080808080808070700FF03FA
:109D0200020504070609080B0A0D0C0F0E111013A9
:109D1200121514FF0055014005259D00CF09950637
:109D220000000044554D500049440050494E470040
:109D32004700474F0044524553455400524553454E
:109D420054005359535F5752004143540041435406
:109D5200494F4E005245475F575200570057520035
:109D620057524954450053594E435F575200535777
:109D7200520043414C550044454300484558004376
:109D8200414C430043414C44000D0A205B4349448B
:109D92003A005D20005245540052455455524E003F
:109DA20052554E0048454C50004C004C544F5353B2
:109DB200005400544F5353004349440054455354F4
:109DC2000043484B0044454D4F004D4F4E49544FC0
:109DD20052004241554400534541524348004C45CC
:109DE20044005343414E0055504441544500440001
:109DF200535445500042414C414E4345004F464664
:109E0200004F4E004E414D4500434F505900500007
:109E1200504147450042004245464F5245004E00E0
:109E22004E45585400474F544F004D4F4E00524537
:109E320000520052440052454144004800455849EE
:109E420054005341560053415645004E4557004D6C
:109E5200004D4952524F520053455400504C415903
:109E6200004900494E534552540044454C4554451F
:089E7200004D4F56450053005E
:00000001FF
